:020000040800F2
:1000000000060020F50500088D24000841240008A2
:10001000692400084124000861240008F70500084D
:10002000F7050008F7050008F70500084D6000080F
:10003000F7050008F7050008F7050008F7050008B0
:10004000F7050008F7050008F7050008F7050008A0
:10005000F7050008F7050008216400084D64000852
:1000600079640008A5640008D1640008F705000859
:10007000F7050008F7050008F7050008F705000870
:10008000F7050008F7050008F7050008F705000860
:10009000F7050008F7050008F7050008FD640008EB
:1000A000F7050008F7050008F7050008F705000840
:1000B000F7050008F7050008F7050008F705000830
:1000C000F7050008F7050008F7050008F705000820
:1000D000F7050008F7050008E9650008F7050008BE
:1000E00061650008F7050008F7050008F705000836
:1000F000F7050008F7050008F7050008F7050008F0
:10010000F7050008F7050008FD650008F705000879
:10011000F7050008F7050008F7050008F7050008CF
:10012000F7050008F7050008F7050008F7050008BF
:10013000F7050008F7050008F7050008F7050008AF
:10014000F7050008F7050008F7050008F70500089F
:10015000F7050008F7050008F7050008F70500088F
:10016000F7050008F7050008F7050008F70500087F
:10017000F705000801580008F7050008F705000812
:10018000F7050008F7050008F7050008F70500085F
:10019000F7050008F7050008F7050008F70500084F
:1001A000F7050008F7050008F7050008F70500083F
:1001B000D5650008F7050008F7050008F7050008F1
:1001C000F7050008F7050008F7050008F70500081F
:1001D000F7050008ED570008F7050008F7050008C7
:1001E000F7050008F7050008F7050008F7050008FF
:1001F000F7050008F7050008F7050008F7050008EF
:10020000F7050008F7050008F7050008F7050008DE
:10021000F7050008F7050008F7050008F7050008CE
:10022000F7050008F70500086D4C0008F705000801
:10023000F7050008F7050008F7050008F7050008AE
:10024000F7050008F7050008F7050008F70500089E
:10025000F7050008F7050008F7050008F70500088E
:10026000F7050008F7050008F7050008F70500087E
:10027000F7050008F7050008F7050008F70500086E
:10028000F7050008F7050008F7050008F70500085E
:10029000F7050008F7050008F7050008F70500084E
:1002A000F7050008F7050008F7050008F70500083E
:1002B000F7050008F7050008F7050008F70500082E
:1002C000F7050008F7050008F7050008F70500081E
:1002D000F7050008F7050008F7050008F70500080E
:1002E000D9070008092100081924000800000000AF
:1002F00053B94AB9002908BF00281CBF4FF0FF318D
:100300004FF0FF3000F074B9ADF1080C6DE904CE88
:1003100000F006F8DDF804E0DDE9022304B07047E0
:100320002DE9F047089D04468E46002B4DD18A42A8
:10033000944669D9B2FA82F252B101FA02F3C2F1DB
:10034000200120FA01F10CFA02FC41EA030E94406C
:100350004FEA1C48210CBEFBF8F61FFA8CF708FB8D
:1003600016E341EA034306FB07F199420AD91CEB65
:10037000030306F1FF3080F01F81994240F21C8197
:10038000023E63445B1AA4B2B3FBF8F008FB1033DF
:1003900044EA034400FB07F7A7420AD91CEB040414
:1003A00000F1FF3380F00A81A74240F207816444E4
:1003B000023840EA0640E41B00261DB1D440002369
:1003C000C5E900433146BDE8F0878B4209D9002DCD
:1003D00000F0EF800026C5E9000130463146BDE857
:1003E000F087B3FA83F6002E4AD18B4202D38242C1
:1003F00000F2F980841A61EB030301209E46002D70
:10040000E0D0C5E9004EDDE702B9FFDEB2FA82F2C4
:10041000002A40F09280A1EB0C014FEA1C471FFA22
:100420008CFE0126200CB1FBF7F307FB131140EA09
:1004300001410EFB03F0884208D91CEB010103F1D6
:10044000FF3802D2884200F2CB804346091AA4B298
:10045000B1FBF7F007FB101144EA01440EFB00FE6C
:10046000A64508D91CEB040400F1FF3102D2A645D1
:1004700000F2BB800846A4EB0E0440EA03409CE770
:10048000C6F12007B34022FA07FC4CEA030C20FA1D
:1004900007F401FA06F31C43F9404FEA1C4900FA3D
:1004A00006F3B1FBF9F8200C1FFA8CFE09FB1811BA
:1004B00040EA014108FB0EF0884202FA06F20BD92D
:1004C0001CEB010108F1FF3A80F08880884240F27D
:1004D0008580A8F102086144091AA4B2B1FBF9F0C1
:1004E00009FB101144EA014100FB0EFE8E4508D9BC
:1004F0001CEB010100F1FF346CD28E456AD9023841
:10050000614440EA0840A0FB0294A1EB0E01A14225
:10051000C846A64656D353D05DB1B3EB080261EB93
:100520000E0101FA07F722FA06F3F1401F43C5E96D
:10053000007100263146BDE8F087C2F12003D840A3
:100540000CFA02FC21FA03F3914001434FEA1C47E5
:100550001FFA8CFEB3FBF7F007FB10360B0C43EAD7
:10056000064300FB0EF69E4204FA02F408D91CEB87
:10057000030300F1FF382FD29E422DD90238634485
:100580009B1B89B2B3FBF7F607FB163341EA034125
:1005900006FB0EF38B4208D91CEB010106F1FF3874
:1005A00016D28B4214D9023E6144C91A46EA00466B
:1005B00038E72E46284605E70646E3E61846F8E6FD
:1005C0004B45A9D2B9EB020864EB0C0E0138A3E746
:1005D0004646EAE7204694E74046D1E7D0467BE727
:1005E000023B614432E7304609E76444023842E79F
:1005F000704700BF02E000F000F8FEE772B637482F
:1006000080F30888364880F3098836483649086000
:1006100040F20000CCF200004EF63471CEF2000140
:100620000860BFF34F8FBFF36F8F40F20000C0F23E
:10063000F0004EF68851CEF200010860BFF34F8FF4
:10064000BFF36F8F4FF00000E1EE100A4EF63C71E1
:10065000CEF200010860062080F31488BFF36F8F8C
:1006600004F06CFA05F05CFC4FF055301F491B4A52
:1006700091423CBF41F8040BFAE71D49184A9142E8
:100680003CBF41F8040BFAE71A491B4A1B4B9A423C
:100690003EBF51F8040B42F8040BF8E7002018495C
:1006A000184A91423CBF41F8040BFAE704F084FA7F
:1006B00005F0A6FC144C154DAC4203DA54F8041BAB
:1006C0008847F9E700F050F8114C124DAC4203DABC
:1006D00054F8041B8847F9E704F06CBA00060020C0
:1006E000002200200000000808ED00E000000020CB
:1006F00000060020506E000800220020C8220020C2
:10070000C8220020B04A0020E0020008EC020008E5
:10071000EC020008EC0200082DE9F04F2DED108AE4
:10072000C1F80CD0D0F80CD0BDEC108ABDE8F08F29
:10073000002383F311882846A047002003F096FB8E
:10074000FEE703F0AFFA00DFFEE70000054B10B54F
:1007500004460360806810B103685B6898472046D0
:1007600010BD00BF5069000870B500F027FD04F00F
:100770000BF9054604F0D8F90446B8B9144B9D426C
:1007800016D001339D4241F2883512BF0446002540
:100790000124104E002004F001F9304601F0D6FA91
:1007A00040B944F6206003F067FBF6E70025F0E768
:1007B0000546EEE70CB100F091F800F0F1FE00F014
:1007C00069FD284600F028F900F088F8F9E700BF35
:1007D000010007B0C82200200448054B054A036009
:1007E00000230549836005F063BF00BFC8220020D5
:1007F00050690008002500204D07000808B500F0EA
:1008000015FDA0F120035842584108BD07B5042149
:1008100001900DEB010000F027FD03B05DF804FB33
:1008200007B541F21203022101A8ADF8043000F02F
:100830001BFD03B05DF804FB38B5302383F311884A
:10084000174803680BB103F0F5FB0023154A4FF47A
:100850007A71134803F0E4FB002383F31188124CF0
:10086000236813B12368013B2360636813B1636895
:10087000013B63600D4D2B7833B963687BB902206F
:1008800000F0CEFD322363602B78032B07D1636821
:100890002BB9022000F0C4FD4FF47A73636038BDB9
:1008A00058230020390800087824002070230020F5
:1008B000084B187003280CD8DFE800F00805020880
:1008C000022000F0A5BD022000F098BD024B0022DE
:1008D0005A6070477023002078240020F7B54648FE
:1008E00001A901F0B3FB002800F08480434B444A87
:1008F0001C46196801317AD004339342F9D16268F9
:10090000404B9A4273D9404B9B6803F1006303F557
:1009100000339A426BD2002000F0E2FC0220FFF785
:10092000C7FF3A4B00219A6C99641A6F19671A6FC6
:10093000DA6CD9645A6F59675A6F1A6D19659A6FD4
:1009400099679B6F324BD3F8802042F00072C3F856
:100950008020D3F8802022F00072C3F88020D3F8E2
:10096000803072B64FF0E023C3F8084DD4E900049C
:10097000BFF34F8FBFF36F8F264AC2F88410BFF3C7
:100980004F8F536923F480335361BFF34F8FD2F8F5
:10099000803043F6E076C3F3C905C3F34E335B0101
:1009A00003EA060C29464CEA81770139C2F87472D1
:1009B000F9D2203B13F1200FF2D1BFF34F8FBFF3D9
:1009C0006F8FBFF34F8FBFF36F8F536923F40033E3
:1009D00053610023C2F85032BFF34F8FBFF36F8FC4
:1009E000302383F31188854680F308882047024826
:1009F00000F074FE03B0F0BDC82200200000020821
:100A000020000208FFFF01080022002000450258D4
:100A10000044025800ED00E02DE9F04FB04B9DB0CE
:100A20002022FF21079014A89E68DB68069300F03F
:100A300061FDAC4A1378A3B90121AB481170036082
:100A4000302383F3118803680BB103F0F3FA00231A
:100A5000A64A4FF47A71A44803F0E2FA002383F324
:100A60001188079B13B1A24B079A1A60A14A137809
:100A7000032B03D0002313709D4A53600023079D6E
:100A80001F469B46CDE90433012000F0C1FC25B18F
:100A9000974B1B68002B00F05783002000F0C6FB2B
:100AA0000C900C9B002BF2DB012000F0A7FC0C9BB0
:100AB000213B1F2BE8D801A252F823F03D0B000880
:100AC000650B0008FB0B0008890A0008890A00086A
:100AD000890A0008A90E0008C3100008650F000865
:100AE00041100008671000088D100008890A0008EE
:100AF0009F100008890A00080B110008DD0B000890
:100B0000890A00084F1100088F0C0008C70D000863
:100B1000890A0008B90F0008890A0008890A000834
:100B2000890A0008890A0008890A0008890A000859
:100B3000890A0008890A0008FB0B00080220FFF759
:100B40005DFE002840F02B83079B0221059A0FA829
:100B5000002A08BF1D4641F21233ADF83C3000F0C8
:100B600083FB91E74FF47A7000F060FB041EEBDB2F
:100B70000220FFF743FE0028E6D0013C052C00F2DE
:100B80001083DFE804F0030A0D1013370523042156
:100B90000FA80F9300F068FB17E004215048F9E715
:100BA00004215548F6E704215448F3E74FF01C08A8
:100BB000404608F1040800F095FB04210F900FA8AF
:100BC00000F052FBB8F12C0FF2D10120049B4FF042
:100BD000000B00FA04F41C43E3B2049300F0D6FCCB
:100BE0002FB1049B03F00B030B2B08BF0025FFF76D
:100BF00017FE49E704214248CCE7002FA4D0049B0C
:100C000003F00B030B2B9FD10220FFF7F7FD0446E7
:100C1000002899D00120002700F062FB0220FFF796
:100C200047FE5FFA87F8404600F06AFB0546B0B120
:100C30000C9940460137A1F140025142514100F068
:100C40006FFB0028EDD10546059441F212130221F5
:100C50000FA82746ADF83C3000F006FB14E72E46FF
:100C60000120FFF725FE1E4B9B68B34207D9304693
:100C700000F038FB013040F097820436F3E700269D
:100C80001C4B274605941E70194B5E60A6E7002F8B
:100C90003FF45AAF049B03F00B030B2B7FF454AFCC
:100CA00064210DA800F0D6FA804600287FF44CAFEE
:100CB0000220FFF7A3FD044600283FF445AFDFF80C
:100CC00048908DF82F80D9F82420D9F8203053434C
:100CD0000D9A93421AD20B4800F0ACFB34E700BFE8
:100CE0000022002074240020582300203908000826
:100CF00078240020702300200422002008220020F5
:100D00000C220020F4670008C8220020BE48474695
:100D1000C24600F08FFBFFF783FD01210DF12F008C
:100D200000F0A2FA0D9B534541D900230EAA394683
:100D30004846CDE90E330FAB00F0D4FC002884D038
:100D400001F0ACFB0E9B00EB030801210DF12F001D
:100D500000F08AFA01F0A2FB404520D9484600F095
:100D6000FBFE80B964210D9BA848013701FB0AF105
:100D7000B1FBF3F18DF82F10C9B200F05BFBD9F88D
:100D800020309A44CEE701F089FB0F9B1844404580
:100D90003FF65BAF01F082FB0E9B00EB03080E9B5E
:100DA0004FF47A70A3FB000303F066F8CDE76423E9
:100DB00001210DF12F0027468DF82F3000F054FA55
:100DC000002306930AE7002F3FF4BEAE049B03F016
:100DD0000B030B2B7FF4B8AE0220FFF769FD322026
:100DE00000F024FA041EFFF6AFAE069BA046E318FF
:100DF0000893874B089ADB689A423FF6A5AEB4F594
:100E0000807F3FF7A1AEDFF80CA24FF000094C4500
:100E10000EDD4FF47A7000F009FA0C900C9B002B59
:100E2000FFF692AE0C9B09F101090AF8013BEEE7CF
:100E3000C820FFF7E3FC044600283FF485AE0027F6
:100E4000DFF8D491CDE90E77B8F1000F02D1274633
:100E5000089BB6E70FAB6F4A0699484602930EAB64
:100E60003A44394401930DAB0093434601F056F8E0
:100E700000283FF4EAAE01F013FB0D9B8A4609906F
:100E80001F44A8EB030801F00BFB099A0E9B9B186B
:100E90004AF10002834272EB0103F4D2484600F0AB
:100EA0005BFE0028EFD1CFE7002F3FF44DAE049B4F
:100EB00003F00B030B2B7FF447AE0220FFF7F8FC87
:100EC000322000F0B3F9B0F10008FFF63DAE18F0A3
:100ED00003047FF439AE4E4A08EB0603926893424E
:100EE0003FF632AEB8F5807F3FF72EAEDFF82491A3
:100EF000A0450DDD4FF47A7000F098F90C900C9B32
:100F0000002BFFF621AE0C9B013409F8013BEFE703
:100F1000C820FFF773FC044600283FF415AE1F2ECF
:100F200011D8C6F1200214AB26F00300394942451E
:100F3000184428BF4246089200F0AAFA089AFF21F6
:100F4000344800F0D7FAC8F38702324930464FEAF6
:100F5000A80900F0D7FA074600283FF476AE06EB62
:100F600089063BE60220FFF749FC00283FF4ECAD80
:100F700000F0F4F900283FF4E7AD0024A046244B2C
:100F80009B68A34258D91F2C11D8149B01330ED053
:100F900024F003031CAA134453F8203C0F9340464B
:100FA00004220FA9043401F0B7F88046E7E7204691
:100FB00000F098F90F90F2E764210EA800F04AF9CA
:100FC000044600287FF4C0AD0220FFF717FC00287C
:100FD0003FF4BAAD0E9BA046DFF83CA003F0030936
:100FE0000E99A1EB0901A14218D9214604230FAAA9
:100FF000504600F0DFFF404604220FA901F08CF8B4
:1010000004348046ECE700BF196800083168000826
:101010000022002074230020C8220020B9F1000F14
:101020000AD04B460FAA624800F0C4FF40464A4629
:101030000FA901F071F880464046FFF7E7FBCDE5C8
:10104000002364210FA80F9300F004F900287FF417
:101050007BAD0220FFF7D2FB00283FF475AD0F985F
:1010600000F072F9E9E7002364210FA80F9300F064
:10107000F1F800287FF468AD0220FFF7BFFB0028DD
:101080003FF462AD0F9800F061F9D6E70220FFF758
:10109000B5FB00283FF458AD00F070F9CDE7022011
:1010A000FFF7ACFB00283FF44FAD0FA9142000F070
:1010B0006BF90890FFF7AAFB08990FA800F0D4F885
:1010C0008CE5322000F0B2F8041EFFF63DADA30718
:1010D0007FF43AAD374A04EB0B03926893423FF634
:1010E00033AD0220FFF78AFB00283FF42DAD24F03A
:1010F00003045C44A3453FF471AD58460BF1040B67
:1011000000F0F0F8FFF782FBF4E74FF47A70FFF796
:1011100075FB00283FF418AD00F020F9002845D0F9
:10112000149B01330BD0082214A9002000F0EAF927
:1011300000283BD02022FF2114A800F0DBF9FFF7A4
:101140006FFB1D4802F098FE1DB0BDE8F08F002F28
:101150003FF4FAAC049B03F00B030B2B7FF4F4ACCD
:10116000002364210FA80F9300F074F804460028B0
:101170007FF4EAAC0220FFF741FB804600283FF4F1
:10118000E3ACFFF74DFB41F2883002F075FE0F989B
:1011900000F048FA4746254600F0F8F974E407469F
:1011A0001CE54FF0000BCFE405944EE53C464CE5C2
:1011B000C822002000220020A08601007047000005
:1011C0002DE9F84F4FF47A7306460D46002402FBD2
:1011D00003F7DFF85080DFF8509098F900305FFA9D
:1011E00084FA5A1C01D0A34212D159F824002A468D
:1011F00031460368D3F820B03B46D847854207D133
:10120000074B012083F800A0BDE8F88F0124E4E734
:10121000002CFBD04FF4FA7002F02EFE0020F3E712
:10122000C42400201022002014220020002307B52F
:10123000024601210DF107008DF80730FFF7C0FFCE
:1012400020B19DF8070003B05DF804FB4FF0FF30BC
:10125000F9E700000A46042108B5FFF7B1FF80F066
:101260000100C0B2404208BD074B0A4630B41978AD
:10127000064B53F82140014623682046DD69044BA4
:10128000AC4630BC604700BFC424002014220020BC
:10129000A086010070B5104C0025104E03F020F917
:1012A00020803068238883420CD8002520880138AC
:1012B00003F012F923880544013BB5F5802F238004
:1012C000F4D370BD03F008F9336805440133B5F574
:1012D000003F3360E5D3E8E7C624002080240020E7
:1012E00003F0DCB900F1006000F5003000687047E1
:1012F00000F10060920000F5003003F053B90000E7
:10130000054B1A68054B1B889B1A834202D910446F
:1013100003F0E2B80020704780240020C62400209B
:1013200038B50446074D29B128682044BDE8384047
:1013300003F0EAB82868204403F0D4F80028F3D07A
:1013400038BD00BF802400200020704700F1FF500E
:1013500000F58F10D0F8000870470000064991F89A
:10136000243033B100230822086A81F82430FFF7C3
:10137000BFBF0120704700BF84240020014B1868C4
:10138000704700BF0010005C194B0138032208446D
:1013900070B51D68174BC5F30B042D0C1E88A642B3
:1013A0000BD15C680A46013C824213460FD214F905
:1013B000016F4EB102F8016BF6E7013A03F1080341
:1013C000ECD181420B4602D22C2203F8012B0424DB
:1013D000094A1688AE4204D1984284BF967803F831
:1013E000016B013C02F10402F3D1581A70BD00BF39
:1013F0000010005C1C2200206C680008022803D149
:10140000024B4FF400129A61704700BF0018025857
:10141000022802D1014B20229A617047001802581D
:10142000022804D1024A536983F0200353617047B4
:10143000001802580FB4124B30B51A78B5B042B943
:101440000122104910481A704FF461430B6001F0FB
:10145000B1FE39AB0C4C389AC82102A8019300F0B8
:10146000EDFF2368C8280246DD6902A9074B28BFA3
:10147000C8222046A84735B0BDE8304004B07047C8
:10148000C8240020CC24002024250020A0860100B0
:10149000002310B5934203D0CC5CC4540133F9E768
:1014A00010BD0000013810B510F9013F3BB191F9B2
:1014B00000409C4203D11AB10131013AF4E71AB15C
:1014C00091F90020981A10BD1046FCE70138013947
:1014D00010F9013F11F9012F0BB19342F8D0981A7E
:1014E0007047000003460246D01A12F9011B00297A
:1014F000FAD1704702440346934202D003F8011B1D
:10150000FAE770472DE9F8431F4D14460746884611
:1015100095F8242052BBDFF870909CB395F82430E6
:101520002BB92022FF2148462F62FFF7E3FF95F8F1
:1015300024004146C0F1080205EB8000A24228BF0A
:101540002246D6B29200FFF7A3FF95F82430A41BE1
:1015500017441E449044E4B2F6B2082E85F8246085
:10156000DBD1FFF7FBFE0028D7D108E02B6A03EBA5
:1015700082038342CFD0FFF7F1FE0028CBD10020B9
:10158000BDE8F8830120FBE784240020024B1A7891
:10159000024B1A70704700BFC424002010220020A4
:1015A00038B51A4C1A4D204601F0A6FE29462046B1
:1015B00001F0CEFE2D681748D5F89020D2F80438F7
:1015C00043F00203C2F8043802F056FC12492846E0
:1015D00001F0CCFFD5F89020104DD2F804382868DF
:1015E00023F002030E49A042C2F804384FF4E1335D
:1015F0000B6001D001F0DEFD6868A04204D008490C
:10160000BDE8384001F0D6BD38BD00BF002C002039
:10161000946B000840420F009C6B000814220020CD
:10162000AC2400200C4B70B50C4D04461E780C4BBE
:1016300055F826209A420DD00A4B00211822184650
:10164000FFF758FF0460014655F82600BDE87040DA
:1016500001F0B0BD70BD00BFC424002014220020E2
:10166000002C0020AC24002080697047C0697047BE
:10167000006A7047406A7047806A7047F0B5ADF203
:10168000044D0E46054600214FF47F7201A80091DB
:10169000FFF730FF2C6A744301362B6A7343A34271
:1016A00016D92B686A46214628465F684FF4806346
:1016B000B84770B16A464FF4806312F8011BFF29E6
:1016C0000AD1013B9BB2002BF7D104F58064E4E71B
:1016D00001200DF2044DF0BD0020FAE78068036898
:1016E000DB69184730B5456A85B004468D420FD393
:1016F0000568CDE90023026A03ABAD6A5143A847F0
:1017000020B1206A039BC31A5842584105B030BD2E
:101710000020FBE7F0B5C56987B004468D4212D3BF
:101720000C9F866905687143CDE9013705AB0093CD
:101730006D69036AA84720B1A069059BC31A584286
:10174000584107B0F0BD0020FBE70000F0B566236C
:1017500089B0002405464FF480768068079403A979
:10176000CDE90336CDE9054403685B699847A8686D
:1017700022462146036800941F692346B847A8689B
:101780009923079403A9CDE90336CDE905440368FD
:101790005B699847A86822462146036800941D6942
:1017A0002346A84709B0F0BD254B2DE9F04F1B7823
:1017B0009FB0002504468DF828304FF09F0E8068BA
:1017C0004FF00123ADF8295005A90995CDE905E3AE
:1017D000CDE9075503685B699847A068032229464D
:1017E000036800922A461E690AABB04730B394F8EA
:1017F0008C200C21134B01FB02339DF828101A7921
:1018000091421BD19DF829205B799A4216D1A0689C
:101810004FF05A0C0C4B082605A90996CDE905C3D3
:10182000CDE9075503685B699847A0682A462946B1
:10183000036800961F690AABB84738B900204BE12E
:10184000DC67000824690008002500010422B34970
:101850000AA804F067FF05460028EFD1BDF82C3038
:101860006FF48277A3813B44012BE7D8079605A943
:10187000CDE90A00A06803685B699847A0682A461A
:101880002946036800961E690AABB0470028D5D0E8
:10189000DDE90A361A0202F4706242EA1662FF2A91
:1018A000CCD11B0E26F07F4650222946142B2661F0
:1018B0000AA828BF1423A373FFF71CFEA06807968D
:1018C00005A903685B699847A068A37B294602685D
:1018D0009B0000930AAB16692A46B0470028ADD09A
:1018E0000B990029AADBC9086FF07E43149D4FF0C5
:1018F000010E994228BF1946C5F303130EFA03F2ED
:1019000021FA03F303916161A261E361002B95D099
:101910002646A44600274FF002081EAAC7F3460336
:1019200002EB830353F834AC07F001031B01DA1D0B
:101930000EFA03F908FA02F2A2EB090202EA0A021D
:10194000DA401AD003F108090F330EFA02F2216AC5
:1019500008FA03F30EFA09FBCCF830208A42A3EB15
:101960000B0B0BEA0A0A2AFA09F98CF82C90A36AE5
:1019700088BF2262934288BFA26201370CF1100C2B
:10198000042FCAD1236A4FF0020C039A4FF0010EC4
:10199000139F9A4224BFB2FBF3F1616207F00F017B
:1019A00038BF01234FF0090201F1010138BF636222
:1019B0004900336B33B3531C0EFA02F8A2F1050948
:1019C0000CFA03F30EFA09FAA3EB080302F1FF384D
:1019D0000CFA08F83B40A8EB0A08D34008EA0708CD
:1019E00028FA09F87BD0012B7BD0022B7BD0032B6C
:1019F00008BF4FF47A735FFA88F808FB0333736308
:101A00004B43B36307321036252AD2D115F0C04FAD
:101A1000C5F3417369D0012B69D0022B0CBF4FF481
:101A20007A634FF47A43C5F3046202FB0333E3663F
:101A30004B432367199B9E075CD0062384F87430C0
:101A400015F4005F05F00F03C5F3042514BF402211
:101A50000822013305FB02255B00A5675D430A9B55
:101A60009F02E5677FF5EAAE0C9BC3F30722C3F341
:101A7000421103F01F0384F8802084F8881084F852
:101A80008130002A3FF4DAAE189BC3F3025213F4FC
:101A9000401F84F883207FF4D1AEDE0602D5042AED
:101AA0007FF4CCAE03F40072002A14BF012200229E
:101AB00084F8872004D0DD0324D5002384F88930FE
:101AC000179B1A0722D5002384F88630702384F8E8
:101AD0008530012384F88D301FB0BDE8F08F0123DD
:101AE00089E7102387E7802385E710239BE74FF4DE
:101AF000807398E7590701D550239FE713F0780FBB
:101B00009ED09BE69903DBD50123D7E75B07E0D5A1
:101B1000012384F886300523D9E700BF7C680008DC
:101B200030B58BB000240546806803924FF0012247
:101B3000059105A9CDE90624CDE90844026852695A
:101B40009047A8680121039B02680091214615690E
:101B50002246A8470BB030BD13B50446A068036801
:101B6000DB6C98470028F9D10DF1070294F8851035
:101B70002046FFF7D5FF94F886309DF807001BB18B
:101B800000F0010002B010BDC043C0F3C010F9E77F
:101B900030B54FF001238BB00024054680688DF8E6
:101BA0000F20059105A9CDE90634CDE90844036865
:101BB0005B699847A86801220DF10F010368009442
:101BC0001D692346A8470BB030BD0000F7B5174686
:101BD0000DF1070206461D46FFF7A2FF68B19DF80A
:101BE000074039469DF82020304624EA05042A4063
:101BF00022438DF80720FFF7CBFF03B0F0BD0000B4
:101C000030B54FF4807389B0002405468068039195
:101C100003A9CDE90434CDE9064403685B6998471C
:101C2000A86822462146036800941D692346A847F8
:101C300009B030BD10B5044623682046DB6A9847DA
:101C40000028F9D110BD000010B590F8743004469A
:101C50005BB1FFF7EFFF012394F87410204684F87E
:101C60008E30BDE81040FFF7CBBF012010BD000053
:101C700010B590F87430044653B1FFF7DBFF012331
:101C80002046042184F88E30BDE81040FFF7B8BF2D
:101C9000012010BDF0B590F883308BB00446042BC2
:101CA00050D100270DF10E0205218DF80E708DF830
:101CB0000F70FFF735FF00282FD00DF10F023521EF
:101CC0002046FFF72DFF40B320461F4EFFF7BCFF15
:101CD0002046FFF7AFFF05AD0FCE0FC5336805A94E
:101CE0009DF80E202B609DF80F30A06843F0020392
:101CF0008DF810208DF80F308DF8113003685B6976
:101D00009847A068022204A9036800971D693B4612
:101D1000A84720B92046FFF7ABFF002010E020467F
:101D2000FFF7A6FF0DF10F0235212046FFF7F8FE61
:101D30000028F2D09DF80F309B07EED50123636099
:101D40000BB0F0BD0120FBE7E06700082DE9F3418F
:101D5000002304468068A36010B103685B6898475D
:101D60000025264E264F0C2301A839465FFA85F838
:101D70006B439A5900F072FA019BA0680022A3609D
:101D8000019210B103685B689847019810B103682D
:101D90005B689847A368E3B141F2883084F88C808F
:101DA00002F06AF82046FFF7D1FC1E2002F064F82A
:101DB0002046FFF7F9FC054688B994F88C300C22D0
:101DC00010485343F158FFF735FB284602B0BDE8F1
:101DD000F0810135032DC6D10B4800F059FB204698
:101DE000FFF758FF0C2294F88C3005465343F15806
:101DF00008B90648E7E70648E5E700BF2469000898
:101E0000E424002084680008FA680008AE6800082E
:101E1000D86800082DE9F041044688B00F46164600
:101E2000FFF712FF2046FFF705FF0025C722A06835
:101E30004FF48073079503A9CDE90323CDE9055538
:101E400003685B699847A0682A462946036800959D
:101E5000D3F810802B46C047054630B92046FFF71F
:101E600007FF284608B0BDE8F081E36E3B60236FB2
:101E70003360F3E72DE9F041002588B01F460446A2
:101E80000E460E9B00F1400CA8463D60016B81B1EF
:101E9000A9420ED391420CD8B6FBF1FE01FB1E61A4
:101EA00039B9416B90F82C800F9D1960816B2960C6
:101EB000154610306045E9D16DB3AB1962699342A4
:101EC00029D82046FFF7C0FE2046FFF7B3FE4FF4A7
:101ED0001453A06803A9CDF80C80CDE90436002680
:101EE000CDE9066603685B699847A06832463146CB
:101EF00003680096D3F810803346C0470646204654
:101F00002EB9FFF7B5FE304608B0BDE8F081FFF707
:101F1000AFFE3D60F7E70026F5E700002DE9F04150
:101F20008669054688B00F46B3429046B1FBF6FC81
:101F300006FB1C1C28BF3346A6EB0C0C00269C4558
:101F4000644628BF1C46FFF77FFE2846FFF772FE57
:101F50000222A86803A9164B0597CDE90323CDE912
:101F6000066603685B699847A8682246414603688D
:101F700000961F693346B847064628462EB9FFF734
:101F800077FE304608B0BDE8F081FFF771FE0E9B8A
:101F90001C60AB6FAA696343B3FBF2F30F9A136043
:101FA000EA6F109B5443AA69B4FBF2F41C60E8E7A3
:101FB000002500012DE9F04FCE18436989B0044691
:101FC0009E420F46914639D83D464FF40458DFF8FB
:101FD00078A0FFF72FFEAE4234D994F88030A6EBFC
:101FE000050B94F8882003A903930023BBF5806FA9
:101FF000A0680693636828BF4FF4806B0595012B9A
:1020000014BF43465346012A049394F8813008BF15
:1020100003F1FF33079303685B699847A068A9EB56
:1020200007030268CDF800B02B44D2F810B00022AC
:102030001146D84718B105F58065CCE7002009B0F6
:10204000BDE8F08F0120FAE700ED0003F0B504468B
:1020500089B00E46FFF7EEFD94F887502DB194F845
:1020600089302BB1012B24D00025284609B0F0BDC2
:1020700094F880300393F02306934FF404530493B1
:102080006368012B04BF1D4B04930023059394F850
:102090008130A06803A9079303685B699847A0682B
:1020A000314603689B6998470546642001F0E4FEC9
:1020B000DBE720460027FFF7C7FD2046FFF7BAFD04
:1020C00008238122852120460097FFF77FFD0546E2
:1020D00018B92046FFF7CCFDC7E794F88030069783
:1020E0000393074B04936368012B04BF054B0493D0
:1020F0000023059394F88130013BCAE700ED00030B
:102100000021001000ED0013014B024A1A607047D5
:10211000E42400204C6A000830B50A44084D91427E
:102120000DD011F8013B5840082340F30004013B57
:102130002C4013F0FF0384EA5000F6D1EFE730BDE6
:102140002083B8ED70470000704700000020704702
:102150000020704713B56C4600F1140384E80600B4
:1021600094E8030083E8050002B010BD002070472A
:1021700013B56C4600F10C0384E8060094E80300F4
:1021800083E8050002B010BD0023C0E903337047A7
:1021900082B002AB03E9060002B07047704700004E
:1021A00000207047704700000020704700207047F3
:1021B0000120704782B0002002A901E90C0002B0A2
:1021C000704700000020704700207047036B1A79A9
:1021D000034B53F832309B699868C0F34010704746
:1021E000E46900080B6883634B6843638B68C363CF
:1021F000CB6803640B6943647047000038B5036B18
:102200000446154D1B7955F8330001F0AFFCD4E9B5
:102210000B231B7955F8331002F1300349689942BA
:1022200018D000231363E26A5363D4E90B12537C82
:10223000581E137C92681B0443EA002313438B63EC
:10224000D4E90B131B79303155F83300BDE8384021
:1022500001F020BC38BD00BFE4690008F8B51D4F8F
:1022600005460E4611463868FFF730F978BB7468AA
:102270003B7924B394F82C209A420BD02468F8E7D9
:102280000122B52100F00EF9736823603B79746078
:1022900084F82C30482004F015FA68B1002202714D
:1022A000C0E90322C0E90522027A42F00702027265
:1022B000094AC0E90B47026028602846F8BD402063
:1022C00004F000FA04460028DAD12C60F5E7002378
:1022D0002B60F2E7EC240020F4690008044B10B5F1
:1022E00004460360406A08B104F0EAF9204610BDD4
:1022F0009869000810B50446FFF7F0FF204604F087
:10230000DDF9204610BD000008B519B1FFF776FFD2
:10231000012008BD036B1A79024B53F8320001F01B
:1023200029FCF5E7E46900082DE9FF41DDF8288084
:102330000546174603911FFA88F60293FFF75EFFE2
:1023400002ABBAB203A9E86A009600F0BFF80446EF
:1023500038B900212846FFF7D7FF204604B0BDE872
:10236000F081AFB92B6B05F134011A79134B53F897
:102370003200B8F1000F19D101F09AFB80F001048E
:10238000E4B23346E86ADDE9022100F0C5F8E0E78F
:10239000029B83B92B6B3A46084805F134011C793E
:1023A000039B50F8340001F099FBE7E7029B42469B
:1023B00001F0AAFBE2E70024E3E700BFE4690008BC
:1023C00013B504460191FFF719FF019A236B04F13D
:1023D00034011879054B53F8300001F0ABFB0021B4
:1023E0002046FFF791FF012002B010BDE46900080C
:1023F00010B50446FFF702FF236B1A79054B53F81B
:10240000320001F0A5FB00212046FFF77DFF0120EF
:1024100010BD00BFE4690008054B064A1A6000229F
:102420001A719A60044ADA6040F21F121A827047E9
:10243000EC2400201B69000800E1F50500F07EBADD
:1024400000B59BB0EFF3098168226846FFF720F8DA
:10245000EFF30583014B9B6BFEE700BF00ED00E04F
:1024600008B5FFF7EDFF000000B59BB0EFF3098161
:1024700068226846FFF70CF8EFF30583014B5B6BAE
:10248000FEE700BF00ED00E0FEE70000FEE7000011
:102490000FB408B5029801F07BFCFEE702F014BA15
:1024A00002F0ECB938B5084B044615460175436097
:1024B0000A21243002F0A6FA04F128002A460A2153
:1024C00002F0A0FA204638BD606A0008F8B51E4642
:1024D0001B6805460C4617461BB9236863B90124DF
:1024E00008E0BDF818203146806A02F0A3FA0028FF
:1024F000F3D100242046F8BD21463A46686A02F02E
:10250000CFFA04460028EAD13368002BF1D0A86A3C
:1025100002F0FAFAEEE7000038B50D46114604461F
:102520001A4611B1806A02F0ADFA2DB12946606AEF
:10253000BDE8384002F0E0BA38BD00000368002171
:102540001B68184703790BB10022027118467047C7
:1025500003685B681847000003791BB90123037106
:1025600018467047002070477047000010B50446B9
:1025700004F0A4F8204610BDF0B500F10B0423468A
:102580000D46B1FBF2F102FB115707F13006392E6F
:10259000C8BF07F13706954203F8016DF0D2421E1D
:1025A000E11A13F8015B9C4202F8015FF9D108447B
:1025B000F0BD00002DE9F04F804687B015464FF082
:1025C00000090C4614F8013B002B3BD0252B08D00A
:1025D000D8F800201946404609F10109D268904711
:1025E00049E14B782D2B06BF8C1C0123002301935E
:1025F00023782B2B06BF01340127002794F800A075
:10260000BAF1300F0CBF01344FF0200A23782A2B87
:102610001CD16178023455F804BB2E2943D12178AE
:1026200081B12A2921D0661C0020A1F13002344654
:10263000D2B2092A1DD80A2316F8011B03FB002079
:102640000029F2D1484607B0BDE8F08F4FF0000BEB
:1026500014F8011B0029F5D0A1F13002D2B2092AE9
:10266000DBD80A2303FB0B2BF2E76178023455F821
:10267000040B01F0DF024C2A17D121780029E1D0A8
:10268000782904F101041FD8622900F20081582939
:102690001AD84E2900F23081442900F0918049294E
:1026A00000F08E8010E00020E3E7A1F141027829DC
:1026B000D2B209D862290BD8582905D84E293BD85F
:1026C000442978D0492976D02E468DF80C1056E052
:1026D000A1F16306152EF7D80FF2040C5CF826F072
:1026E00071270008B7270008C9260008C926000876
:1026F000C9260008C9260008B7270008C92600080F
:10270000C9260008C9260008C9260008C9260008ED
:102710004728000835290008C9260008C9260008EE
:1027200087270008C926000831290008C9260008A3
:10273000C926000835290008A1F14F02092AC3D88B
:1027400001A050F822F000BF4728000835290008F2
:10275000C9260008C9260008C9260008C92600089D
:1027600031290008C9260008C926000835290008B3
:102770002E464FF0200A56F8042B8DF80C2003AD9E
:102780000DF10D002BE02E4647F6FF726A4B56F80E
:10279000045B002808BF1046002D08BF1D462A46CE
:1027A0002F18104612F8011B11B1B91A0029F8DAD6
:1027B0004FF0200A13E02E46192A56F8041B02D8BF
:1027C0002E4656F8041B002936DA2D2249428DF890
:1027D0000C200DF10D000A2203ADFFF7CDFE471BC3
:1027E0000199ABEB070323EAE372002945D1002BE3
:1027F000C2F1000B1EDD29782D2901D02B290DD126
:10280000BAF1300F0AD1D8F800304046019209F1F0
:102810000109DB68013F98470135019AD8F800307B
:10282000514640460192DB6898471BF1010B019A23
:10283000F4D191443B4615E01FB12B228DF80C20BA
:10284000C7E703A8C7E708222E4603A856F8041BCB
:10285000C2E7D8F80020404615F8011BD268019362
:102860009047019B013BF4D5002FA8BFB9445D46BA
:102870002DB9D94435462146A3E69346DAE7D8F880
:10288000003051464046013DDB689847F0E7A1F132
:102890006302152A3FF618AF01A353F822F000BFD8
:1028A00071270008C1270008C9260008C9260008AA
:1028B000C9260008C9260008C1270008C926000843
:1028C000C9260008C9260008C9260008C92600082C
:1028D0004728000835290008C9260008C92600082D
:1028E00087270008C926000831290008C9260008E2
:1028F000C926000835290008A1F14F02092A3FF630
:10290000E3AE01A353F822F0472800083529000858
:10291000C9260008C9260008C9260008C9260008DB
:1029200031290008C9260008C926000835290008F1
:102930000A2289E7102287E7786A0008F0B5054681
:1029400087B016461F460C4689B14A1E0023294609
:1029500001A800F05FF83A46314601A8FFF72AFEC9
:10296000049BA3423CBF0022EA5407B0F0BD0A46D4
:10297000ECE70000D0E902239A421FBF4268D1541D
:10298000C36801331ABFC36000206FF001007047B5
:10299000D0E903239A421FBF4268D25C013303612E
:1029A00014BF10466FF001007047000003692BB19F
:1029B000013B426803610020D15470476FF0010071
:1029C0007047000038B504460846D4E903315B1A65
:1029D000934228BF13461D4663682A461944FEF7F2
:1029E00057FD236928462B44236138BD38B504467A
:1029F000D0E902301B1A934228BF13461D46636874
:102A00002A461844FEF744FDE36828462B44E36059
:102A100038BD000010B5C0E90223034C0023C0E913
:102A20000041036110BD00BF806A00088A0710B52D
:102A300004461DD50378042B1AD143681B682BB1BB
:102A40000522027098472378052B01D102232370B9
:102A5000302383F31188002104F1080001F026FAE5
:102A6000002383F31188E069BDE8104002F0BCB98F
:102A7000CB0704D50248BDE8104001F089B910BD6C
:102A8000986A000810B5044C204600F0FBFF034A8A
:102A90000023C4E9062310BD042500200050005285
:102AA00010B503780446012B12D10E4B98420FD17A
:102AB00002460D49102002F069F90C4BE0615A6B97
:102AC00042F480425A63DA6D42F48042DA65DB6D8B
:102AD0006268A36992685A60054A1A601B22DA602C
:102AE00010BD00BF042500202D2A00080045025813
:102AF0001500020182691B2310B5D360D1E90030B3
:102B000013F44C4406D19B011461D06103F440439B
:102B1000536110BD0024184313F4406F1461CC6856
:102B2000D4615061F5D08B689361F2E730B5846968
:102B30001B25C069E5600068836104F12003C3615F
:102B400002234261013A03614223C3601623836278
:102B5000CB682261E361D1E90023134312F4406F93
:102B6000636101D08B68A361C36843F00103C36054
:102B700030BD000030B5D0E90640006804F1200502
:102B80008561C36108234261013A036146230D69EF
:102B9000C36016238362CB682261E361D1E900231D
:102BA000134312F4406F43EA854343F0806363614B
:102BB00001D08B68A361C36843F00103C36030BDDB
:102BC0008069036823F0040310B5CC680360002318
:102BD0000361C4618361D1E900430969234343EA86
:102BE000814343F04063436112B14FF010431360DF
:102BF00010BD000083691A6842F002021A601A6868
:102C00009207FCD41A6842F004021A607047000070
:102C10008269936810B5D3609B0704461DD503787D
:102C2000032B1AD143681B682BB105220270984709
:102C30002378052B01D102232370302383F31188DD
:102C4000002104F1080001F031F9002383F3118819
:102C5000E069BDE8104002F0C7B810BD02684368E3
:102C60001143016003B1184770470000024A13681E
:102C700043F0C003136070470044004013B50E4C8E
:102C8000204600F08BFA04F1140000234FF4007288
:102C90000A49009400F048F9094B4FF400720949C1
:102CA00004F13800009400F0C1F9074A074BC4E969
:102CB000172302B010BD00BF24250020902500205E
:102CC0006D2C0008902700200044004000E1F5052D
:102CD000037C30B5214C002918BF0C46012B0CD1C8
:102CE0001F4B984209D11F4B9A6C42F400329A64F0
:102CF0001A6F42F400321A671B6F2268036EC16DAF
:102D000003EB52038466B3FBF2F36268150442BF1F
:102D100023F0070503F0070343EA4503CB60A368EC
:102D200043F040034B60E36843F001038B6042F4DF
:102D3000967343F001030B604FF0FF330B625105B4
:102D400005D512F0102205D0B2F1805F04D080F8D2
:102D5000643030BD7F23FAE73F23F8E7A86A000814
:102D600024250020004502582DE9F047C66D054690
:102D70003768F469210734621AD014F0080118BFCB
:102D80004FF48071E20748BF41F02001A3074FF0E4
:102D9000300348BF41F04001600748BF41F0800167
:102DA00083F31188281DFFF759FF002383F311884F
:102DB000E2050AD5302383F311884FF48061281D82
:102DC000FFF74CFF002383F311884FF030094FF0D9
:102DD000000A14F0200838D13B0616D54FF0300910
:102DE00005F1380A200610D589F31188504600F005
:102DF00051F9002836DA0821281DFFF72FFF27F0A8
:102E000080033360002383F31188790614D56206AA
:102E100012D5302383F31188D5E913239A4208D1C0
:102E20002B6C33B127F040071021281DFFF716FF48
:102E30003760002383F31188E30618D5AA6E13695F
:102E4000ABB15069BDE8F047184789F31188736A40
:102E5000284695F86410194000F0BAF98AF31188F1
:102E6000F469B6E7B06288F31188F469BAE7BDE89F
:102E7000F0870000F8B51546826804460B46AA4262
:102E800000D28568A1692669761AB5420BD2184628
:102E90002A46FEF7FDFAA3692B44A3612846A368DE
:102EA0005B1BA360F8BD0CD9AF1B18463246FEF77A
:102EB000EFFA3A46E1683044FEF7EAFAE3683B4449
:102EC000EBE718462A46FEF7E3FAE368E5E7000079
:102ED00083689342F7B50446154600D28568D4E965
:102EE0000460361AB5420BD22A46FEF7D1FA63695E
:102EF0002B4463612846A3685B1BA36003B0F0BD4D
:102F00000DD93246AF1B0191FEF7C2FA01993A463C
:102F1000E0683144FEF7BCFAE3683B44E9E72A463F
:102F2000FEF7B6FAE368E4E710B50A440024C3618B
:102F3000029B8460C16002610362C0E90000C0E9D5
:102F4000051110BD08B5D0E90532934201D1826860
:102F500082B98268013282605A1C42611970002174
:102F6000D0E904329A4224BFC368436100F0B8FF3D
:102F7000002008BD4FF0FF30FBE7000070B53023A4
:102F800004460E4683F31188A568A5B1A368A2691B
:102F9000013BA360531CA36115782269934224BFAF
:102FA000E368A361E3690BB120469847002383F3EC
:102FB0001188284607E03146204600F081FF0028AE
:102FC000E2DA85F3118870BD2DE9F74F04460E460D
:102FD00017469846D0F81C904FF0300A8AF31188B3
:102FE0004FF0000B154665B12A4631462046FFF7E3
:102FF00041FF034660B94146204600F061FF0028CA
:10300000F1D0002383F31188781B03B0BDE8F08F63
:10301000B9F1000F03D001902046C847019B8BF304
:103020001188ED1A1E448AF31188DCE7C160C36180
:10303000009B82600362C0E905111144C0E90000F1
:1030400001617047F8B504460D461646302383F3F8
:103050001188A768A7B1A368013BA36063695A1CE4
:1030600062611D70D4E904329A4224BFE36863614F
:10307000E3690BB120469847002080F3118807E0F0
:103080003146204600F01CFF0028E2DA87F3118861
:10309000F8BD0000D0E9052310B59A4201D182683D
:1030A0007AB982680021013282605A1C82611C78E0
:1030B00003699A4224BFC368836100F011FF204670
:1030C00010BD4FF0FF30FBE72DE9F74F04460E46E9
:1030D00017469846D0F81C904FF0300A8AF31188B2
:1030E0004FF0000B154665B12A4631462046FFF7E2
:1030F000EFFE034660B94146204600F0E1FE00289D
:10310000F1D0002383F31188781B03B0BDE8F08F62
:10311000B9F1000F03D001902046C847019B8BF303
:103120001188ED1A1E448AF31188DCE702684368AF
:103130001143016003B11847704700001430FFF7D6
:1031400043BF00004FF0FF331430FFF73DBF0000D6
:103150003830FFF7B9BF00004FF0FF333830FFF7CA
:10316000B3BF00001430FFF709BF00004FF0FF317C
:103170001430FFF703BF00003830FFF763BF0000D3
:103180004FF0FF323830FFF75DBF0000012914BF58
:103190006FF0130000207047FFF770BD044B036011
:1031A00000234360C0E9023301230374704700BF6A
:1031B000C06A000810B53023044683F31188FFF776
:1031C00087FD02230020237480F3118810BD0000C6
:1031D00038B5C36904460D461BB904210844FFF7FE
:1031E000A5FF294604F11400FFF7ACFE002806DA1B
:1031F000201D4FF40061BDE83840FFF797BF38BD90
:10320000026843681143016003B11847704700002A
:1032100013B5406B00F58054D4F8A4381A681178BF
:10322000042914D1017C022911D1197901231289B1
:103230008B4013420BD101A94C3002F029FCD4F889
:10324000A4480246019B2179206800F0DFF902B012
:1032500010BD0000143002F0ABBB00004FF0FF3394
:10326000143002F0A5BB00004C3002F07DBC000021
:103270004FF0FF334C3002F077BC0000143002F006
:1032800079BB00004FF0FF31143002F073BB000037
:103290004C3002F049BC00004FF0FF324C3002F0DD
:1032A00043BC00000020704710B500F58054D4F8EE
:1032B000A4381A681178042917D1017C022914D185
:1032C0005979012352898B4013420ED1143002F0F8
:1032D0000BFB024648B1D4F8A4484FF4407361791F
:1032E0002068BDE8104000F07FB910BD406BFFF7CB
:1032F000DBBF0000704700007FB5124B012504269C
:10330000044603600023057400F1840243602946EB
:10331000C0E902330C4B0290143001934FF4407318
:10332000009602F0BDFA094B04F69442294604F1D6
:103330004C000294CDE900634FF4407302F084FB2B
:1033400004B070BDE86A0008ED32000811320008D0
:103350000A68302383F311880B790B3342F823007A
:103360004B79133342F823008B7913B10B3342F8B6
:10337000230000F58053C3F8A4180223037400202F
:1033800080F311887047000038B5037F044613B1FD
:1033900090F85430ABB90125201D0221FFF730FF12
:1033A00004F114006FF00101257700F0A5FD04F190
:1033B0004C0084F854506FF00101BDE8384000F033
:1033C0009BBD38BD10B5012104460430FFF718FF3E
:1033D0000023237784F8543010BD000038B504462C
:1033E0000025143002F074FA04F14C00257702F045
:1033F00043FB201D84F854500121FFF701FF2046B4
:10340000BDE83840FFF750BF90F8803003F060030C
:10341000202B06D190F881200023212A03D81F2ACF
:1034200006D800207047222AFBD1C0E91D3303E0F3
:10343000034A426707228267C3670120704700BFC3
:103440003422002037B500F58055D5F8A4381A6825
:10345000117804291AD1017C022917D11979012385
:1034600012898B40134211D100F14C04204602F026
:10347000C3FB58B101A9204602F00AFBD5F8A448C5
:103480000246019B2179206800F0C0F803B030BDEE
:1034900001F10B03F0B550F8236085B004460D46EA
:1034A000FEB1302383F3118804EB8507301D08211A
:1034B000FFF7A6FEFB6806F14C005B691B681BB1B9
:1034C000019002F0F3FA019803A902F0E1FA024632
:1034D00048B1039B2946204600F098F8002383F367
:1034E000118805B0F0BDFB685A691268002AF5D052
:1034F0001B8A013B1340F1D104F18002EAE700008E
:10350000133138B550F82140ECB1302383F31188E2
:1035100004F58053D3F8A4281368527903EB82038F
:10352000DB689B695D6845B104216018FFF768FEA0
:10353000294604F1140002F0E1F92046FFF7B4FE39
:10354000002383F3118838BD7047000001F09EBC52
:1035500001234022002110B5044600F8303BFDF75E
:10356000C9FF0023C4E9013310BD000010B53023AA
:10357000044683F311882422416000210C30FDF7BA
:10358000B9FF204601F0A4FC02230020237080F341
:10359000118810BD70B500EB8103054650690E46D9
:1035A0001446DA6018B110220021FDF7A3FFA069CC
:1035B00018B110220021FDF79DFF31462846BDE8D5
:1035C000704001F085BD000083682022002103F0D7
:1035D000011310B5044683601030FDF78BFF2046C1
:1035E000BDE8104001F000BEF0B4012500EB8104FD
:1035F00047898D40E4683D43A469458123600023E9
:10360000A2606360F0BC01F01DBE0000F0B40125B3
:1036100000EB810407898D40E4683D4364690581BE
:1036200023600023A2606360F0BC01F093BE000041
:1036300070B5022300250446242203702946C0F8F1
:1036400088500C3040F8045CFDF754FF204684F8A5
:10365000705001F0D1FC63681B6823B129462046F5
:10366000BDE87040184770BD0378052B10B50446BF
:103670000AD080F88C300523037043681B680BB1B7
:10368000042198470023A36010BD0000017805299C
:1036900006D190F88C20436802701B6803B118476C
:1036A0007047000070B590F87030044613B10023E5
:1036B00080F8703004F18002204601F0B9FD6368A3
:1036C0009B68B3B994F8803013F0600535D00021C1
:1036D000204602F0ABF80021204602F09BF8636818
:1036E0001B6813B1062120469847062384F87030E2
:1036F00070BD204698470028E4D0B4F88630A26F09
:103700009A4288BFA36794F98030A56F002B4FF0D1
:10371000300380F20381002D00F0F280092284F84A
:10372000702083F3118800212046D4E91D23FFF780
:103730006DFF002383F31188DAE794F8812003F00A
:103740007F0343EA022340F20232934200F0C58035
:1037500021D8B3F5807F48D00DD8012B3FD0022B64
:1037600000F09380002BB2D104F18802626702223C
:10377000A267E367C1E7B3F5817F00F09B80B3F5F3
:10378000407FA4D194F88230012BA0D1B4F88830C6
:1037900043F0020332E0B3F5006F4DD017D8B3F514
:1037A000A06F31D0A3F5C063012B90D86368204689
:1037B00094F882205E6894F88310B4F88430B0479F
:1037C000002884D0436863670368A3671AE0B3F5F1
:1037D000106F36D040F6024293427FF478AF5C4BD4
:1037E00063670223A3670023C3E794F88230012BA9
:1037F0007FF46DAFB4F8883023F00203A4F888306A
:10380000C4E91D55E56778E7B4F88030B3F5A06FDB
:103810000ED194F88230204684F88A3001F04AFCB8
:1038200063681B6813B10121204698470323237066
:103830000023C4E91D339CE704F18B036367012374
:10384000C3E72378042B10D1302383F3118820465B
:10385000FFF7BAFE85F311880321636884F88B5063
:1038600021701B680BB12046984794F88230002BDA
:10387000DED084F88B300423237063681B68002B30
:10388000D6D0022120469847D2E794F884302046CB
:103890001D0603F00F010AD501F0BCFC012804D07D
:1038A00002287FF414AF2B4B9AE72B4B98E701F0DB
:1038B000A3FCF3E794F88230002B7FF408AF94F870
:1038C000843013F00F01B3D01A06204602D501F060
:1038D000C5FFADE701F0B6FFAAE794F88230002BF0
:1038E0007FF4F5AE94F8843013F00F01A0D01B06DE
:1038F000204602D501F09AFF9AE701F08BFF97E787
:10390000142284F8702083F311882B462A46294616
:103910002046FFF769FE85F31188E9E65DB11522BF
:1039200084F8702083F3118800212046D4E91D23F8
:10393000FFF75AFEFDE60B2284F8702083F311880E
:103940002B462A4629462046FFF760FEE3E700BFE4
:10395000186B0008106B0008146B000838B590F85D
:1039600070300446002B3ED0063BDAB20F2A34D822
:103970000F2B32D8DFE803F03731310822323131F2
:103980003131313131313737856FB0F886309D4272
:1039900014D2C3681B8AB5FBF3F203FB12556DB951
:1039A000302383F311882B462A462946FFF72EFE43
:1039B00085F311880A2384F870300EE0142384F80C
:1039C0007030302383F31188002320461A461946AD
:1039D000FFF70AFE002383F3118838BDC36F03B1DC
:1039E00098470023E7E70021204601F01FFF002150
:1039F000204601F00FFF63681B6813B106212046C3
:103A000098470623D7E7000010B590F870300446B9
:103A1000142B29D017D8062B05D001D81BB110BD07
:103A2000093B022BFBD80021204601F0FFFE0021BC
:103A3000204601F0EFFE63681B6813B106212046A3
:103A40009847062319E0152BE9D10B2380F8703035
:103A5000302383F3118800231A461946FFF7D6FD59
:103A6000002383F31188DAE7C3689B695B68002B46
:103A7000D5D1C36F03B19847002384F87030CEE7E7
:103A8000FFF700B8012100230170C0E901330C30B9
:103A900000F028B910B53023044683F31188416043
:103AA000FEF7FEFF02230020237080F3118810BD73
:103AB00010B53023044683F31188032304F8083B30
:103AC000FFF718F84FF0FF31204600F0E1F900232E
:103AD00083F31188C01A18BF012010BD38B5044601
:103AE000302585F31188032504F8085BFFF71EF8DD
:103AF0004FF0FF31204600F0CBF9002383F311880B
:103B0000C01A18BF012038BD38B50446302585F3EA
:103B10001188042504F8085BFFF72CF84FF0FF31FB
:103B2000204600F0B5F9002383F31188C01A18BFAE
:103B3000012038BD10B53023044683F31188FFF708
:103B40003FF806232370002383F3118810BD000083
:103B500010B53023044683F31188FFF74BF8022396
:103B60002370002383F3118810BD00000C3000F097
:103B7000D5B800000C3000F0DBB8000000238268EC
:103B8000037503691B6899689142FBD25A68036008
:103B900042601060586070470023826803750369B3
:103BA0001B6899689142FBD85A68036042601060B4
:103BB0005860704708B50846302383F311880A7DA2
:103BC0000023052A06D8DFE802F00B050503120ED4
:103BD000826913604FF0FF338361FFF7CFFF00234B
:103BE00083F3118808BD8269936801339360D0E93B
:103BF000003213605A60EDE7FFF7C0BF054BD9688C
:103C000008751868026853601A600122D86002754E
:103C1000FCF782BD902900200C4B30B5DD684B1CB1
:103C200087B004460FD02B46094A684600F0F8F9E1
:103C30002046FFF7E3FF009B13B1684600F0FAF956
:103C4000A86907B030BDFFF7D9FFF9E79029002038
:103C5000B53B000838B50C4D04468161EB688168BE
:103C60009A68914203D8BDE83840FFF787BF1846ED
:103C7000FFF792FF01230146EC6020462375BDE863
:103C80003840FCF749BD00BF90290020044B1A685A
:103C9000DB6890689B68984294BF002001207047C1
:103CA00090290020084B10B51C68D8682268536022
:103CB0001A600122DC602275FFF76EFF0146204684
:103CC000BDE81040FCF728BD90290020044B1A687D
:103CD000DB6892689B689A4201D9FFF7E3BF70479F
:103CE00090290020C0E90000816070478368013B93
:103CF000002B10B583600CDA074BDC684368A061C9
:103D0000206063601C6044600520FFF777FFA069B6
:103D100010BD0020FCE700BF9029002008B530232B
:103D200083F31188FFF7E2FF002383F3118808BDB6
:103D300008B5302383F3118883680133002B836037
:103D400007DC036800211A68026050601846FFF71C
:103D500081FF002383F3118808BD000038B50123DB
:103D6000084C00252370656001F082FF01F0A8FF78
:103D70000549064802F07CF80223237085F3118878
:103D800038BD00BFF82B0020206B000890290020D0
:103D900008B572B6044B186500F062FD00F030FE05
:103DA000024B03221A70FEE790290020F82B002016
:103DB00000F076B9EFF3118020B9EFF305833022DC
:103DC00082F311887047000010B530B9EFF3058415
:103DD000C4F3080414B180F3118810BDFFF776FF17
:103DE00084F31188F9E70000034A516853685B1AAD
:103DF0009842FBD8704700BF001000E08B600223A0
:103E0000086108468B8270478368A3F1840243F8F7
:103E1000142C026943F8442C426943F8402C094AA7
:103E200043F8242CC268A3F1200043F8182C022286
:103E300003F80C2C002203F80B2C034A43F8102C37
:103E4000704700BF310700089029002008B5FFF730
:103E5000DBFFBDE80840FFF7CFBE0000024BDB6888
:103E600098610F20FFF7CABE90290020302383F30A
:103E70001188FFF7F3BF000008B50146302383F334
:103E800011880820FFF7C8FE002383F3118808BDBE
:103E9000054BDB6821B1036098610320FFF7BCBECE
:103EA0004FF0FF30704700BF9029002003682BB10E
:103EB0000022026018469961FFF79EBE704700001D
:103EC000064BDB6839B1426818605A601360436082
:103ED0000420FFF7A1BE4FF0FF307047902900206B
:103EE0000368984206D01A680260506018469961CB
:103EF000FFF782BE7047000038B504460D462068C3
:103F0000844200D138BD036823605C608561FFF79F
:103F100073FEF4E7036810B59C68A2420CD85C6895
:103F20008A600B604C602160596099688A1A9A60B7
:103F30004FF0FF33836010BD121B1B68ECE70000DD
:103F40000A2938BF0A2170B504460D460A266019B1
:103F500001F088FE01F070FE041BA54203D8751C19
:103F600004462E46F3E70A2E04D90120BDE870402E
:103F700001F0BEBF70BD0000F8B5144B0D460A2A13
:103F80004FF00A07D96103F11001826038BF0A229D
:103F9000416019691446016048601861A81801F071
:103FA00051FE01F049FE431B0646A34206D37C1C8A
:103FB00028192746354601F055FEF2E70A2F04D9A5
:103FC0000120BDE8F84001F093BFF8BD9029002022
:103FD000F8B506460D4601F02FFE0F4A134653F87A
:103FE000107F9F4206D12A4601463046BDE8F84080
:103FF000FFF7C2BFD169BB68441A2C1928BF2C46F1
:10400000A34202D92946FFF79BFF224631460348C7
:10401000BDE8F840FFF77EBF90290020A0290020CE
:10402000C0E90323002310B45DF8044B4361FFF79C
:10403000CFBF000010B5194C236998420DD081689C
:10404000D0E9003213605A609A680A449A600023EB
:1040500003604FF0FF33A36110BD0268234643F8AD
:10406000102F53600022026022699A4203D1BDE8FA
:10407000104001F0F1BD936881680B44936001F03A
:10408000DBFD2269E1699268441AA242E4D9114435
:10409000BDE81040091AFFF753BF00BF9029002068
:1040A0002DE9F047DFF8BC8008F110072C4ED8F856
:1040B000105001F0C1FDD8F81C40AA68031B9A42B9
:1040C0003ED814444FF00009D5E90032C8F81C402E
:1040D00013605A60C5F80090D8F81030B34201D18F
:1040E00001F0BAFD89F31188D5E9033128469847D4
:1040F000302383F311886B69002BD8D001F09CFD2D
:104100006A69A0EB040982464A450DD2022001F0FB
:10411000EFFE0022D8F81030B34208D151462846AD
:10412000BDE8F047FFF728BF121A2244F2E712EB6E
:1041300009092946384638BF4A46FFF7EBFEB5E77E
:10414000D8F81030B34208D01444C8F81C00211A23
:10415000A960BDE8F047FFF7F3BEBDE8F08700BFF8
:10416000A02900209029002000207047FEE70000D1
:10417000704700004FF0FF307047000002290CD05C
:10418000032904D00129074818BF00207047032ADB
:1041900005D8054800EBC20070470448704700206E
:1041A000704700BFF86B000844220020AC6B000889
:1041B00070B59AB005460846144601A900F0C2F849
:1041C00001A8FDF78FF9431C0022C6B25B00104620
:1041D000C5E9003423700323023404F8013C01AB29
:1041E000D1B202348E4201D81AB070BD13F8011B4F
:1041F000013204F8010C04F8021CF1E708B5302381
:1042000083F311880348FFF71DF9002383F3118816
:1042100008BD00BF002C002090F8803003F01F0282
:10422000012A07D190F881200B2A03D10023C0E98D
:104230001D3315E003F06003202B08D1B0F8843063
:104240002BB990F88120212A03D81F2A04D8FFF720
:10425000DBB8222AEBD0FAE7034A426707228267DB
:10426000C3670120704700BF3B22002007B5052926
:1042700017D8DFE801F0191603191920302383F34A
:104280001188104A01210190FFF784F90198022159
:104290000D4AFFF77FF90D48FFF7A0F8002383F3DD
:1042A000118803B05DF804FB302383F311880748BD
:1042B000FFF76AF8F2E7302383F311880348FFF72A
:1042C00081F8EBE74C6B0008706B0008002C0020B5
:1042D00038B50C4D0C4C2A460C4904F10800FFF788
:1042E00067FF05F1CA0204F110000949FFF760FFFA
:1042F00005F5CA7204F118000649BDE83840FFF719
:1043000057BF00BFD8440020442200202C6B000877
:10431000366B0008416B000870B5044608460D4630
:10432000FDF7E0F8C6B22046013403780BB9184611
:1043300070BD32462946FDF7B5F80028F3D10120BB
:10434000F6E700002DE9F04705460C46FDF7CAF8F0
:104350002B49C6B22846FFF7DFFF08B10736F6B291
:1043600028492846FFF7D8FF08B11036F6B2632E69
:104370000BD8DFF88C80DFF88C90234FDFF894A007
:104380002E7846B92670BDE8F08729462046BDE85C
:10439000F04702F01BBA252E2ED1072241462846AF
:1043A000FDF780F870B9194B224603F10C0153F860
:1043B000040B8B4242F8040BF9D11B8807350E34ED
:1043C0001380DDE7082249462846FDF76BF898B9C7
:1043D000A21C0F4B197802320909C95D02F8041CAE
:1043E00013F8011B01F00F015345C95D02F8031CCE
:1043F000F0D118340835C3E7013504F8016BBFE785
:10440000186C0008416B00082F6C0008206C000835
:1044100000E8F11F0CE8F11FBFF34F8F044B1A693E
:104420005107FCD1D3F810215207F8D1704700BFD3
:104430000020005208B50D4B1B78ABB9FFF7ECFF1D
:104440000B4BDA68D10704D50A4A5A6002F1883268
:104450005A60D3F80C21D20706D5064AC3F80421C6
:1044600002F18832C3F8042108BD00BF364700209E
:10447000002000522301674508B5114B1B78F3B9A2
:10448000104B1A69510703D5DA6842F04002DA602E
:10449000D3F81021520705D5D3F80C2142F0400281
:1044A000C3F80C21FFF7B8FF064BDA6842F00102AF
:1044B000DA60D3F80C2142F00102C3F80C2108BDE8
:1044C00036470020002000520F289ABF00F5806078
:1044D00040040020704700004FF400307047000097
:1044E000102070470F2808B50BD8FFF7EDFF00F537
:1044F00000330268013204D104308342F9D1012033
:1045000008BD0020FCE700000F2870B5054645D81F
:10451000FFF750FC224CFFF77FFF0646FFF78AFFAC
:104520004FF0FF33072D6361C4F8143120D82361A5
:10453000FFF772FF2B0243F02403E360E36843F0CC
:104540008003E36023695A07FCD42846FFF764FF21
:104550004FF40031FFF7B8FF00F02EFA3046FFF7B6
:104560008BFFFFF731FC2846BDE87040FFF7BABF6C
:10457000C4F81031FFF750FFA5F108031B0243F008
:104580002403C4F80C31D4F80C3143F08003C4F890
:104590000C31D4F810315B07FBD4D6E7002070BD96
:1045A000002000522DE9F84F40EA020305460C4670
:1045B0001746D80602D00020BDE8F88F27F01F0765
:1045C000DFF8D4B0FFF736FF2744BC4203D1012007
:1045D000FFF752FFF0E720222946204602F0A2F81A
:1045E00010B920352034F0E72B4605F120021E6873
:1045F000711CE0D104339A42F9D1FFF7DBFB05F1DE
:104600007843234AB3F5801F224B28BF9A4603F113
:10461000040338BF9046A2F1080228BF9846A3F1D0
:1046200008033ABF9146DA469946FFF7F5FEC8F807
:104630000060A5EB040CD9F8002004F11C0142F045
:104640000202C9F80020221FDAF8006016F0050601
:10465000FAD152F8043F8A424CF80230F4D1BFF349
:104660004F8FFFF7D9FE4FF0FF32C8F80020D9F87E
:10467000002022F00202C9F80020FFF7A5FB20224B
:104680002146284602F04EF80028AAD030469FE77F
:1046900014200052102100521020005210B5084C76
:1046A000237828B11BB9FFF7C5FE0123237010BD85
:1046B000002BFCD02070BDE81040FFF7DDBE00BF2E
:1046C000364700202DE9F04F0D4685B0814658B1A0
:1046D00011F00D0614BF2022082211F008030193E7
:1046E00004D0431E03426AD0002435E0002E37D0A8
:1046F00009F11F0121F01F094FF00108324F05F0A9
:104700000403DFF8D0A005EA080BBBF1000F32D09C
:104710007869C0072FD408F101080C37B8F1060FEB
:10472000F3D19EB9294D4946A819019201F0EAFA40
:10473000044600283AD11836019A782EF3D149461A
:1047400001F0E0FA0446002830D1019A4946204899
:1047500001F0D8FA044668BB204605B0BDE8F08FEA
:104760000029C9D101462846029201F0CBFA04463D
:10477000E0B9029AC0E713B178694107CBD5AC071D
:1047800002D578698007C6D5019911B1786901070A
:10479000C1D51820494600FB08A0CDE9022301F04D
:1047A000B1FA0446DDE902230028B4D04A460021CC
:1047B000204601E04A460021FCF79CFECCE7024679
:1047C000002E95D198E700BF406C00086847002094
:1047D00038470020504700200021FFF773BF00003A
:1047E0000121FFF76FBF0000F8B5144D0124182711
:1047F000134E40F2FF3200210120FCF77BFE07FB45
:10480000046001342A6955F80C1F01F067FA062C80
:10481000F5D137254FF4C0542046FFF7E1FF01469C
:1048200028B122460748BDE8F84001F057BAC4EB6A
:10483000C404013D4FEAD404EED1F8BD406C000839
:1048400050470020384700200421FFF73BBF0000FD
:104850004843FFF7C1BF000008B101F0C5BA704777
:1048600038B5054D00240334696855F80C0B00F089
:10487000B5F8122CF7D138BD406C000870B5104E59
:1048800082B0FFF797FA054601F0D6F93268034681
:104890009042336037BF0B4A0A495168146836BFEB
:1048A0000131D1E9004151600419284641F100016C
:1048B0000191FFF789FA2046019902B070BD00BF4F
:1048C000E0470020E847002070B5124E82B0FFF7A5
:1048D00071FA054601F0B0F9326803469042336040
:1048E00037BF0D4A0C495168146836BF0131D1E910
:1048F000004151600419284641F100010191FFF780
:1049000063FA4FF47A72002320460199FBF7F0FC1A
:1049100002B070BDE0470020E84700200244074B8A
:10492000D2B210B5904200D110BD441C00B253F871
:10493000200041F8040BE0B2F4E700BF50400058FB
:104940000E4B30B51C6F240405D41C6F1C671C6F04
:1049500044F400441C670A4C02442368D2B243F476
:1049600080732360074B904200D130BD441C51F846
:10497000045B00B243F82050E0B2F4E70044025870
:10498000004802585040005807B5012201A90020F4
:10499000FFF7C4FF019803B05DF804FB13B50446AC
:1049A000FFF7F2FFA04205D0012201A900200194E7
:1049B000FFF7C6FF02B010BD0144BFF34F8F064B97
:1049C000884204D3BFF34F8FBFF36F8F7047C3F894
:1049D0005C022030F4E700BF00ED00E00144BFF3CB
:1049E0004F8F064B884204D3BFF34F8FBFF36F8FB7
:1049F0007047C3F870022030F4E700BF00ED00E01C
:104A00007047000070B5054616460C46012010217F
:104A1000FFF71EFF286046733CB1204636B1FFF712
:104A200013FF2B68186000B19C6070BDFFF7D8FEC3
:104A3000F7E7000070B50E461546044600B30B6854
:104A400043608368934210D213B10068FFF704FFFC
:104A5000637B28462BB1FFF7F7FE206020B9A060EA
:104A600070BDFFF7BDFEF8E7A560206805F11F01E6
:104A7000306021F01F01FFF79FFF01202073EFE757
:104A80000120EDE710B5044640B10068884205D129
:104A9000606808B1FCF7FCFC0023237310BD000024
:104AA00070B50E461546044620B383689A4210D965
:104AB00013B10068FFF7D0FE637B28462BB1FFF7E8
:104AC000C3FE206020B9A06070BDFFF789FEF8E743
:104AD000A560316819B12A462068FCF7D9FC206826
:104AE00005F11F01306021F01F01FFF777FF012062
:104AF0002073E9E70120E7E720B103688B4204BF98
:104B0000002303737047000008B10023037370474C
:104B1000034B1A681AB9034AD2F8D0241A607047B6
:104B2000F04700200040025808B5FFF7F1FF024BA4
:104B30001868C0F3806008BDF047002070B5BFF36F
:104B40004F8FBFF36F8F1A4A0021C2F85012BFF384
:104B50004F8FBFF36F8F536943F400335361BFF33B
:104B60004F8FBFF36F8FC2F88410BFF34F8FD2F80F
:104B7000803043F6E074C3F3C900C3F34E335B01E6
:104B800003EA0406014646EA81750139C2F860521B
:104B9000F9D2203B13F1200FF2D1BFF34F8F5369AD
:104BA00043F480335361BFF34F8FBFF36F8F70BDFA
:104BB00000ED00E0FEE70000214B2248224A70B5DC
:104BC000904237D3214BC11EDA1C121A22F0030285
:104BD0008B4238BF00220021FCF78CFC1C4A0023CA
:104BE000C2F88430BFF34F8FD2F8803043F6E074C0
:104BF000C3F3C900C3F34E335B0103EA0406014665
:104C000046EA81750139C2F86C52F9D2203B13F1A2
:104C1000200FF2D1BFF34F8FBFF36F8FBFF34F8FD2
:104C2000BFF36F8F0023C2F85032BFF34F8FBFF333
:104C30006F8F70BD53F8041B40F8041BC0E700BF22
:104C4000186F0008B04A0020B04A0020B04A002087
:104C500000ED00E003681A6899685A6043681BB168
:104C600042EA014180681847704700004FF0A443B2
:104C700010B51C68E00702D52848FFF7EBFFA10735
:104C800002D52748FFF7E6FF620702D52548FFF760
:104C9000E1FF230702D52448FFF7DCFFE00602D539
:104CA0002248FFF7D7FFA10602D52148FFF7D2FF20
:104CB000620602D51F48FFF7CDFF230602D51E4826
:104CC000FFF7C8FFE00502D51C48FFF7C3FFA105A9
:104CD00002D51B48FFF7BEFF620502D51948FFF752
:104CE000B9FF230502D51848FFF7B4FFE00402D549
:104CF0001648FFF7AFFFA10402D51548FFF7AAFF3A
:104D0000620402D51348FFF7A5FF230402D5124819
:104D1000FFF7A0FFBDE8104001F0D0B9F847002030
:104D200004480020104800201C480020284800208B
:104D300034480020404800204C48002058480020BB
:104D400064480020704800207C48002088480020EB
:104D500094480020A0480020AC48002030B5094B02
:104D60000021094C10200725196054F8042B013844
:104D7000C3E90121D16003F10C0311615560F4D145
:104D800030BD00BFF4470020886C00080F28F0B544
:104D90000AD9102806D10F230020114C01272568BD
:104DA000984203D9002018E00346F6E707FA00F618
:104DB000354213D10C23354343432560181D23444A
:104DC000C3E90212074B20445A6B42F001025A63B6
:104DD000DA6D42F00102DA65DB6DF0BD0130DFE72C
:104DE000F4470020004502580368D968DA68C9070B
:104DF00022F03F02DA6002D51A689207FCD507223A
:104E00005A607047054B996B21EA000199631A6E4D
:104E100022EA00021A661B6E704700BF0045025866
:104E200070B5D0E9244300224FF0FF359E6804EBB3
:104E300042135101D3F80009002805DAD3F800091C
:104E400040F08040C3F80009D3F8000B002805DAD1
:104E5000D3F8000B40F08040C3F8000B0132631818
:104E60009642C3F80859C3F8085BE0D24FF001132B
:104E7000C4F81C3870BD0000890141F020010161B7
:104E800003699B06FCD41220FEF7AEBF10B50A4C96
:104E90002046FEF75DFB094BC4F89030084BC4F880
:104EA0009430084C2046FEF753FB074BC4F8903073
:104EB000064BC4F8943010BDB848002000000840EC
:104EC000EC6C00085449002000000440F86C000815
:104ED00070B503780546012B58D13F4BD0F8904070
:104EE000984254D13D4B0E2165209A6B42F00062EE
:104EF0009A631A6E42F000621A661B6E384BD3F842
:104F0000802042F00062C3F88020D3F8802022F095
:104F10000062C3F88020D3F8803000F0ABFC314B46
:104F2000E360314BC4F800380023D5F89060C4F832
:104F3000003EC02323604FF40413A3633369002BA6
:104F4000FCDA01230C203361FEF74EFF3369DB07E7
:104F5000FCD41220FEF748FF3369002BFCDA002650
:104F60002846A660FFF75CFF6B68C4F81068DB6832
:104F7000C4F81468C4F81C6863BB1C4BA3614FF0F1
:104F8000FF336361A36843F00103A36070BD184B56
:104F90009842C9D1114B4FF080609A6B42F0007279
:104FA0009A631A6E42F000721A661B6E0C4BD3F8AD
:104FB000802042F00072C3F88020D3F8802022F0D5
:104FC0000072C3F88020D3F88030FFF71BFF0E215A
:104FD0004D20A2E7074BD1E7B84800200045025812
:104FE000004402584014004003002002003C30C03E
:104FF00054490020083C30C0F8B5D0F89040054630
:1050000000214FF000662046FFF736FFD5F89410D8
:1050100000234FF001128F684FF0FF30C4F834388E
:10502000C4F81C2804EB431201339F42C2F8006904
:10503000C2F8006BC2F80809C2F8080BF2D20B687C
:10504000D5F89020C5F89830636210231361166973
:1050500016F01006FBD11220FEF7C6FED4F8003879
:1050600023F4FE63C4F80038A36943F4402343F0FB
:105070001003A3610923C4F81038C4F814380B4B8B
:10508000EB604FF0C043C4F8103B094BC4F8003B41
:10509000C4F81069C4F80039D5F8983003F110024B
:1050A00043F48013C5F89820A362F8BDC86C0008CB
:1050B00040800010D0F8902090F88A10D2F8003884
:1050C00023F4FE6343EA0113C2F80038704700007E
:1050D0002DE9F84300EB8103D0F890500C46804650
:1050E000DA680FFA81F94801166806F00306731EA4
:1050F000022B05EB41134FF0000194BFB604384E6C
:10510000C3F8101B4FF0010104F1100398BF06F122
:10511000805601FA03F3916998BF06F5004600290D
:105120003AD0578A04F15801374349016F50D5F8F6
:105130001C180B430021C5F81C382B180127C3F895
:105140001019A7405369611E9BB3138A928B9B0869
:10515000012A88BF5343D8F89820981842EA03439D
:1051600001F140022146C8F89800284605EB82026A
:105170005360FFF781FE08EB8900C3681B8A43EA8E
:10518000845348341E4364012E51D5F81C381F4304
:10519000C5F81C78BDE8F88305EB4917D7F8001B64
:1051A00021F40041C7F8001BD5F81C1821EA0303BD
:1051B000C0E704F13F030B4A2846214605EB830371
:1051C0005A60FFF759FE05EB4910D0F8003923F477
:1051D0000043C0F80039D5F81C3823EA0707D7E7A1
:1051E0000080001000040002D0F894201268C0F87B
:1051F0009820FFF715BE00005831D0F890304901D3
:105200005B5813F4004004D013F4001F0CBF0220BD
:10521000012070474831D0F8903049015B5813F4B1
:10522000004004D013F4001F0CBF0220012070477F
:1052300000EB8101CB68196A0B6813604B685360FF
:105240007047000000EB810330B5DD68AA69136880
:10525000D36019B9402B84BF402313606B8A146854
:10526000D0F890201C4402EB4110013C09B2B4FB81
:10527000F3F46343033323F0030343EAC44343F0EB
:10528000C043C0F8103B2B6803F00303012B0ED181
:10529000D2F8083802EB411013F4807FD0F8003BBD
:1052A00014BF43F0805343F00053C0F8003B02EBBF
:1052B0004112D2F8003B43F00443C2F8003B30BD3A
:1052C0002DE9F041D0F8906005460C4606EB4113FD
:1052D000D3F8087B3A07C3F8087B08D5D6F814380A
:1052E0001B0704D500EB8103DB685B689847FA076E
:1052F0001FD5D6F81438DB071BD505EB8403D96816
:10530000CCB98B69488A5A68B2FBF0F600FB1622CA
:105310008AB91868DA6890420DD2121AC3E90024DB
:10532000302383F3118821462846FFF78BFF84F34F
:105330001188BDE8F081012303FA04F26B8923EAA6
:1053400002036B81CB68002BF3D021462846BDE8D1
:10535000F041184700EB81034A0170B5DD68D0F8D1
:1053600090306C692668E66056BB1A444FF4002002
:10537000C2F810092A6802F00302012A0AB20ED10B
:10538000D3F8080803EB421410F4807FD4F8000926
:1053900014BF40F0805040F00050C4F8000903EB07
:1053A0004212D2F8000940F00440C2F8000901227C
:1053B000D3F8340802FA01F10143C3F8341870BD80
:1053C00019B9402E84BF4020206020681A442E8ADC
:1053D0008419013CB4FBF6F440EAC44040F00050AC
:1053E000C6E700002DE9F843D0F8906005460C466A
:1053F0004F0106EB4113D3F8088918F0010FC3F8E9
:1054000008891CD0D6F81038DB0718D500EB8103CB
:10541000D3F80CC0DCF81430D3F800E0DA68964515
:1054200030D2A2EB0E024FF000091A60C3F80490CC
:10543000302383F31188FFF78DFF89F3118818F06B
:10544000800F1DD0D6F834380126A640334217D03D
:1054500005EB84030134D5F89050D3F80CC0E4B2C6
:105460002F44DCF8142005EB0434D2F800E0516836
:10547000714514D3D5F8343823EA0606C5F83468E4
:10548000BDE8F883012303FA01F2038923EA02034A
:105490000381DCF80830002BD1D09847CFE7AEEB82
:1054A0000103BCF81000834228BF0346D7F818094F
:1054B00080B2B3EB800FE3D89068A0F1040959F8EB
:1054C000048FC4F80080A0EB09089844B8F1040FD9
:1054D000F5D818440B4490605360C8E72DE9F84FA5
:1054E000D0F8905004466E69AB691E4016F480589F
:1054F0006E6103D0BDE8F84FFEF79AB8002E12DABD
:10550000D5F8003E9B0705D0D5F8003E23F00303F5
:10551000C5F8003ED5F80438204623F00103C5F84D
:105520000438FEF7B3F8370505D52046FFF778FCB9
:105530002046FEF799F8B0040CD5D5F8083813F0DA
:10554000060FEB6823F470530CBF43F4105343F47D
:10555000A053EB6031071BD56368DB681BB9AB69EF
:1055600023F00803AB612378052B0CD1D5F8003E5E
:105570009A0705D0D5F8003E23F00303C5F8003E96
:105580002046FEF783F86368DB680BB12046984736
:10559000F30200F1BA80B70226D5D4F89090002724
:1055A0004FF0010A09EB4712D2F8003B03F4402305
:1055B000B3F5802F11D1D2F8003B002B0DDA6289B0
:1055C0000AFA07F322EA0303638104EB8703DB682B
:1055D000DB6813B13946204698470137D4F8943038
:1055E000FFB29B689F42DDD9F00619D5D4F8900030
:1055F000026AC2F30A1702F00F0302F4F012B2F5C6
:10560000802F00F0CA80B2F5402F09D104EB83034C
:10561000002200F58050DB681B6A974240F0B080A2
:105620003003D5F8185835D5E90303D500212046B5
:10563000FFF746FEAA0303D501212046FFF740FEEF
:105640006B0303D502212046FFF73AFE2F0303D553
:1056500003212046FFF734FEE80203D5042120464B
:10566000FFF72EFEA90203D505212046FFF728FEED
:105670006A0203D506212046FFF722FE2B0203D53E
:1056800007212046FFF71CFEEF0103D50821204625
:10569000FFF716FE700340F1A780E90703D500214C
:1056A0002046FFF79FFEAA0703D501212046FFF7FA
:1056B00099FE6B0703D502212046FFF793FE2F07C3
:1056C00003D503212046FFF78DFEEE0603D5042106
:1056D0002046FFF787FEA80603D505212046FFF7E1
:1056E00081FE690603D506212046FFF77BFE2A06C8
:1056F00003D507212046FFF775FEEB0574D520463C
:105700000821BDE8F84FFFF76DBED4F890904FF038
:10571000000B4FF0010AD4F894305FFA8BF79B68C6
:105720009F423FF638AF09EB4713D3F8002902F444
:105730004022B2F5802F20D1D3F80029002A1CDAAC
:10574000D3F8002942F09042C3F80029D3F8002989
:10575000002AFBDB3946D4F89000FFF78DFB228945
:105760000AFA07F322EA0303238104EB8703DB68C9
:105770009B6813B13946204698470BF1010BCAE7E5
:10578000910701D1D0F80080072A02F101029CBFE5
:1057900003F8018B4FEA18283FE704EB830300F579
:1057A0008050DA68D2F818C0DCF80820DCE9001C68
:1057B000A1EB0C0C00218F4208D1DB689B699A6831
:1057C0003A449A605A683A445A6029E711F0030F44
:1057D00001D1D0F800808C4501F1010184BF02F8AD
:1057E000018B4FEA1828E6E7BDE8F88F08B50348B3
:1057F000FFF774FEBDE8084000F060BCB848002028
:1058000008B50348FFF76AFEBDE8084000F056BC43
:1058100054490020D0F8903003EB4111D1F8003BFF
:1058200043F40013C1F8003B70470000D0F89030FB
:1058300003EB4111D1F8003943F40013C1F80039EA
:1058400070470000D0F8903003EB4111D1F8003BD5
:1058500023F40013C1F8003B70470000D0F89030EB
:1058600003EB4111D1F8003923F40013C1F80039DA
:1058700070470000090100F16043012203F5614314
:10588000C9B283F8001300F01F039A4043099B003C
:1058900003F1604303F56143C3F880211A60704748
:1058A00030B50433039C0172002104FB0325C16061
:1058B000C0E90653049B0363059BC0E90000C0E9EF
:1058C0000422C0E90842C0E90A11436330BD000068
:1058D0000022416AC260C0E90411C0E90A226FF0E7
:1058E0000101FEF709BB0000D0E90432934201D167
:1058F000C2680AB9181D7047002070470369196013
:105900000021C2680132C260C269134482699342B5
:10591000036124BF436A0361FEF7E2BA38B5044667
:105920000D46E3683BB162690020131D1268A36253
:105930001344E36207E0237A33B929462046FEF791
:10594000BFFA0028EDDA38BD6FF00100FBE7000078
:10595000C368C269013BC3604369134482699342CF
:10596000436124BF436A436100238362036B03B135
:105970001847704770B53023044683F31188866A50
:105980003EB9FFF7CBFF054618B186F311882846CC
:1059900070BDA36AE26A13F8015B9342A36202D36B
:1059A0002046FFF7D5FF002383F31188EFE70000BF
:1059B0002DE9F84F04460E46174698464FF0300939
:1059C00089F311880025AA46D4F828B0BBF1000F4E
:1059D00009D141462046FFF7A1FF20B18BF3118882
:1059E0002846BDE8F88FD4E90A12A7EB050B521A36
:1059F000934528BF9346BBF1400F1BD9334601F1B5
:105A0000400251F8040B914243F8040BF9D1A36A08
:105A1000403640354033A362D4E90A239A4202D388
:105A20002046FFF795FF8AF31188BD42D8D289F34B
:105A30001188C9E730465A46FBF72AFDA36A5E443F
:105A40005D445B44A362E7E710B5029C0433017236
:105A500003FB0421C460C0E906130023C0E90A3334
:105A6000039B0363049BC0E90000C0E90422C0E972
:105A70000842436310BD0000026A6FF00101C2607A
:105A8000426AC0E904220022C0E90A22FEF734BAC1
:105A9000D0E904239A4201D1C26822B9184650F8CD
:105AA000043B0B60704700231846FAE7C3680021E7
:105AB000C2690133C36043691344826993424361FD
:105AC00024BF436A4361FEF70BBA000038B50446B1
:105AD0000D46E3683BB1236900201A1DA262E2690A
:105AE0001344E36207E0237A33B929462046FEF7E0
:105AF000E7F90028EDDA38BD6FF00100FBE70000A0
:105B000003691960C268013AC260C26913448269BC
:105B10009342036124BF436A036100238362036BE2
:105B200003B118477047000070B530230D46044696
:105B3000114683F31188866A2EB9FFF7C7FF10B1AB
:105B400086F3118870BDA36A1D70A36AE26A0133EF
:105B50009342A36204D3E16920460439FFF7D0FFE2
:105B6000002080F31188EDE72DE9F84F04460D463B
:105B7000904699464FF0300A8AF311880026B346C2
:105B8000A76A4FB949462046FFF7A0FF20B187F327
:105B900011883046BDE8F88FD4E90A073A1AA8EB15
:105BA0000607974228BF1746402F1BD905F140032F
:105BB00055F8042B9D4240F8042BF9D1A36A4036D6
:105BC0004033A362D4E90A239A4204D3E169204610
:105BD0000439FFF795FF8BF311884645D9D28AF334
:105BE0001188CDE729463A46FBF752FCA36A3D44AB
:105BF0003E443B44A362E5E7D0E904239A4217D12F
:105C0000C3689BB1836A8BB1043B9B1A0ED01360AF
:105C1000C368013BC360C3691A4483699A42026145
:105C200024BF436A0361002383620123184670473F
:105C30000023FBE700F06CBA014B586A704700BFC5
:105C4000000C0040034B002258631A610222DA6004
:105C5000704700BF000C0040014B0022DA60704723
:105C6000000C0040014B5863704700BF000C00401F
:105C7000024B034A1A60034A5A607047084A0020E0
:105C8000B04A002000000220074B494210B55C6872
:105C9000201A08401968821A8A4203D3A24201D806
:105CA0005A6010BD0020FCE7084A002008B53023E8
:105CB00083F31188FFF7E8FF002383F3118808BD01
:105CC00004480121044B03600023C0E901330C3078
:105CD000FEF708B8104A0020AD5C0008CB1D083A5A
:105CE00023F00703591A521A012110B4D2080024D4
:105CF000C0E9004384600C301C605A605DF8044BBE
:105D0000FDF7F0BF2DE9F84F364ECD1D0F460028A8
:105D100018BF0646082A4FEAD50538BF082206F103
:105D20000C08341D91464046FDF7F8FF09F10701C4
:105D3000C9F1000E224624686CB94046FDF7F8FF11
:105D40003368CBB308224946E8009847044698B325
:105D500040E9026730E004EB010CD4F804A00CEA3F
:105D60000E0C0AF10100ACF1080304EBC0009842EC
:105D7000E0D9A0EB0C0CB5EBEC0F4FEAEC0BD9D84B
:105D80009C421CD204F10802AB45A3EB02024FEA8D
:105D9000E202626009D9691CED43206803EBC1028D
:105DA0005D44556043F8310022601C465F60404608
:105DB00044F8086BFDF7BCFF2046BDE8F88FAA4504
:105DC000216802D111602346EFE7013504EBC503DA
:105DD00044F8351003F10801401AC01058601360F0
:105DE000F1E700BF104A0020F8B550F8043C044623
:105DF00050F8085CA0F1080607332F1D0C35DB08AE
:105E000040F8043C2846FDF789FF3B469F421A684C
:105E100001D0B34228D20AB1964225D244F8082CC8
:105E200054F8042C1E60013254F8081C06EBC20022
:105E3000814206D14868024444F8042C0A6844F8B8
:105E4000082C5868411C03EBC1018E4207D154F85D
:105E5000042C013202445A6054F8082C1A60284677
:105E6000BDE8F840FDF764BF1346CFE7FEE700004A
:105E700070B51B4B0025044686B058600E468562FF
:105E8000016300F0F3F804F11003A560E562C4E9D2
:105E900004334FF0FF33C4E90044C4E90635FFF78B
:105EA000CBFE2B46024604F134012046C4E9082308
:105EB00080230C4A2565FDF7A1FF01230A4AE06013
:105EC00000920375684672680192B268CDE90223B8
:105ED000064BCDE90435FDF7B9FF06B070BD00BF34
:105EE000F82B0020046D0008096D00086D5E0008A5
:105EF000024AD36A1843D062704700BF902900203D
:105F00004B6843608B688360CB68C3600B694361F7
:105F10004B6903628B6943620B6803607047000042
:105F200008B5324B40F2FF70196C014319649A6E48
:105F300002432F489A662F4A9B6E1146FFF7E0FFF7
:105F400000F5806002F11C01FFF7DAFF00F58060C8
:105F500002F13801FFF7D4FF00F5806002F154012F
:105F6000FFF7CEFF00F5806002F17001FFF7C8FF78
:105F700000F5806002F18C01FFF7C2FF00F5806040
:105F800002F1A801FFF7BCFF00F5806002F1C40137
:105F9000FFF7B6FF00F5806002F1E001FFF7B0FF08
:105FA00000F5806002F1FC01FFF7AAFF02F58C7199
:105FB00000F58060FFF7A4FF00F06CF90E4BD3F8FA
:105FC000902242F00102C3F89022D3F8942242F0CA
:105FD0000102C3F894220522C3F898204FF06052C2
:105FE000C3F89C20054AC3F8A02008BD004502580C
:105FF00000000258106D000800ED00E01F000803CB
:1060000008B500F033FBFDF7A9FE0D4BDA6B42F04B
:106010004002DA635A6E22F040025A665B6E094B08
:106020001A6842F008021A601A6842F004021A6004
:10603000FEF76EFDFEF7D8FBBDE80840FEF748B955
:10604000004502580018024870470000EFF309832A
:10605000054968334A6B22F001024A6383F30988D9
:10606000002383F31188704700EF00E0302080F3B5
:10607000118862B60D4B0E4AD96821F4E06109041B
:10608000090C0A430B49DA60D3F8FC2042F0807215
:10609000C3F8FC20084AC2F8B01F116841F00101A2
:1060A00011602022DA7783F82200704700ED00E0CB
:1060B0000003FA0555CEACC5001000E0302310B542
:1060C00083F311880E4B5B6813F4006314D0F1EE78
:1060D000103AEFF309844FF08073683CE361094B99
:1060E000DB6B236684F30988FDF7D0FD10B1064B06
:1060F000A36110BD054BFBE783F31188F9E700BFEF
:1061000000ED00E000EF00E043070008460700084C
:106110000E4B9A6C42F008029A641A6F42F0080221
:106120001A670B4A1B6FD36B43F00803D363C72274
:10613000084B9A624FF0FF32DA6200229A615A638A
:10614000DA605A6001225A611A60704700450258AD
:106150000010005C000C0040094A08B51169D368C2
:106160000B40D9B29B076FEA0101116107D53023BB
:1061700083F31188FDF71CFE002383F3118808BD0B
:10618000000C0040044BDA6B0243DA635A6E104392
:1061900058665B6E704700BF0045025808B53C4B1F
:1061A0004FF0FF31D3F8802062F00042C3F8802026
:1061B000D3F8802002F00042C3F88020D3F880207A
:1061C000D3F88420C3F88410D3F884200022C3F8C5
:1061D0008420D3F88400D86F40F0FF4040F4FF00E3
:1061E00040F4DF4040F07F00D867D86F20F0FF40D8
:1061F00020F4FF0020F4DF4020F07F00D867D86F44
:10620000D3F888006FEA40506FEA5050C3F8880016
:10621000D3F88800C0F30A00C3F88800D3F88800D8
:10622000D3F89000C3F89010D3F89000C3F89020F2
:10623000D3F89000D3F89400C3F89410D3F89400E6
:10624000C3F89420D3F89400D3F89800C3F89810BA
:10625000D3F89800C3F89820D3F89800D3F88C00AE
:10626000C3F88C10D3F88C00C3F88C20D3F88C00C2
:10627000D3F89C00C3F89C10D3F89C10C3F89C2062
:10628000D3F89C30FEF76AFDBDE8084000F0BEB9C7
:106290000044025808B50122504BC3F80821504B66
:1062A0005A6D42F002025A65DA6F42F00202DA6772
:1062B0000422DB6F4B4BDA605A689104FCD54A4AE2
:1062C0001A6001229A60494ADA6000221A614FF48A
:1062D00040429A61434B9A699204FCD51A6842F491
:1062E00080721A60424B1A6F12F4407F04D04FF450
:1062F00080321A6700221A671A6842F001021A6097
:106300003B4B1A685007FCD500221A611A6912F03B
:106310003802FBD1012119604FF0804159605A6762
:10632000344ADA62344A1A611A6842F480321A60D6
:106330002F4B1A689103FCD51A6842F480521A60F8
:106340001A689204FCD52D4A2D499A6200225A639C
:10635000196301F57C01DA6301F5E77199635A6409
:10636000284A1A64284ADA621A6842F0A8521A6067
:106370001F4B1A6802F02852B2F1285FF9D1482267
:106380009A614FF48862DA6140221A621F4ADA6425
:106390001F4A1A651F4A5A651F4A9A6532231F4AC7
:1063A0001360136803F00F03022BFAD1104A13692C
:1063B00043F003031361136903F03803182BFAD178
:1063C0004FF00050FFF7DEFE4FF08040FFF7DAFE9F
:1063D0004FF00040BDE80840FFF7D4BE00800051F8
:1063E000004502580048025800C000F004000001B7
:1063F000004402580000FF0100889008322060002D
:1064000063020901470E0508DD0BBF0120000020D3
:10641000000001100910E0000001011000200052EE
:106420004FF0B04208B5D2F8883003F00103C2F84B
:10643000883023B1044A13680BB150689847BDE80F
:106440000840FFF73BBE00BF284A00204FF0B04293
:1064500008B5D2F8883003F00203C2F8883023B1BF
:10646000044A93680BB1D0689847BDE80840FFF72D
:1064700025BE00BF284A00204FF0B04208B5D2F830
:10648000883003F00403C2F8883023B1044A13694A
:106490000BB150699847BDE80840FFF70FBE00BF39
:1064A000284A00204FF0B04208B5D2F8883003F0F7
:1064B0000803C2F8883023B1044A93690BB1D0694C
:1064C0009847BDE80840FFF7F9BD00BF284A002003
:1064D0004FF0B04208B5D2F8883003F01003C2F88C
:1064E000883023B1044A136A0BB1506A9847BDE85B
:1064F0000840FFF7E3BD00BF284A00204FF0B0433B
:1065000010B5D3F8884004F47872C3F88820A30645
:1065100004D5124A936A0BB1D06A9847600604D535
:106520000E4A136B0BB1506B9847210604D50B4AEA
:10653000936B0BB1D06B9847E20504D5074A136CF7
:106540000BB1506C9847A30504D5044A936C0BB16A
:10655000D06C9847BDE81040FFF7B0BD284A002036
:106560004FF0B04310B5D3F8884004F47C42C3F830
:106570008820620504D5164A136D0BB1506D9847FB
:10658000230504D5124A936D0BB1D06D9847E004F2
:1065900004D50F4A136E0BB1506E9847A10404D571
:1065A0000B4A936E0BB1D06E9847620404D5084A2B
:1065B000136F0BB1506F9847230404D5044A936FAF
:1065C0000BB1D06F9847BDE81040FFF777BD00BF13
:1065D000284A002008B50348FCF71AFBBDE808402C
:1065E000FFF76CBD0425002008B50348FCF7BCFB91
:1065F000BDE80840FFF762BD2425002008B5FFF77D
:10660000ABFDBDE80840FFF759BD0000062108B505
:106610000846FFF72FF906210720FFF72BF906217F
:106620000820FFF727F906210920FFF723F90621A3
:106630000A20FFF71FF906211720FFF71BF9062193
:106640002820FFF717F909217A20FFF713F90A210B
:106650005C20FFF70FF907213220FFF70BF90C211F
:106660002620BDE80840FFF705B9000008B5FFF790
:1066700095FD00F00FF8FCF78FFDFCF767FFFCF7C6
:1066800039FEFDF7FDF9FFF7DFFCBDE80840FFF735
:10669000D1BA00000023054A19460133102BC2E984
:1066A000001102F10802F8D1704700BF284A00200B
:1066B0000B460146184600F027B80000FEF7CCB89C
:1066C000FFF7FCBF012838BF012010B50446204663
:1066D000FEF782F830B900F007F808B900F00CF8BE
:1066E0008047F4E710BD0000024B1868BFF35B8FD2
:1066F000704700BFA84A002008B5062000F04AF8FD
:106700000120FDF733FD000010B5054C13462CB1F8
:106710000A4601460220AFF3008010BD2046FCE788
:106720000000000010B501390244904201D1002060
:1067300005E0037811F8014FA34201D0181B10BDEA
:106740000130F2E71F2938B504460D4604D9162357
:1067500003604FF0FF3038BD426C12B152F8213067
:106760004BB9204600F030F82A4601462046BDE8E5
:10677000384000F017B8012B0AD0591C03D116235A
:1067800003600120E7E7002442F8254028469847A7
:106790000020E0E7024B01461868FFF7D3BF00BFB7
:1067A0006422002038B5074D0023044608461146F0
:1067B0002B60FDF7DFFC431C02D12B6803B1236083
:1067C00038BD00BFAC4A0020FDF7CEBC034611F82F
:1067D000012B03F8012B002AF9D1704700000000BB
:1067E00001000000000100010000000000000000A6
:1067F0000000000052657175657374656420746FE4
:10680000206572617365206D6F7265207468616EBA
:106810002077652063616E0A0045726173652043CD
:106820006F6D6D616E642052656365697665640A9B
:106830000050435420444F4E453A2025640A00003E
:1068400053544D333248373F3F3F0053544D33325A
:10685000483733782F3732780053544D3332483726
:1068600034332F3735332F373530000001105A00BD
:10687000031059000120580003205600534644508D
:10688000000000004A454445433A204661696C6572
:106890006420746F2064657465637420666C617332
:1068A00068206465766963653A2025730A004A4565
:1068B0004445433A204661696C656420746F2063E7
:1068C0006F6E66696720666C6173682064657669BF
:1068D00063653A2025730A004A454445433A2044FB
:1068E0006574656374656420466C617368204465F3
:1068F000766963653A2025730A0045787420466CF2
:10690000617368204E6F7420466F756E64210000BD
:106910006D74323571007732357100773235712DF3
:10692000647472001069000820BA000000000000C2
:1069300016690008EF400000000000001B69000815
:10694000EF700000000000000000000000000000E8
:106950004D1D0008B51F0008691600086D160008D7
:10696000151700081D1F000871160008751600088D
:10697000151E0008E5160008751E0008591B0008C2
:106980007D160008791600084D200008DD16000865
:1069900000000000000000000000000000000000F7
:1069A000452100088924000889240008492100089D
:1069B0004D210008512100085521000889240008B4
:1069C00089240008892400086D210008712100082D
:1069D00089210008912100089D210008A1210008BB
:1069E000A52100080425002001000000000000008F
:1069F00000000000DD220008F52200084521000803
:106A0000B121000829230008E5210008C12300085E
:106A1000F123000855210008C9210008B52100080C
:106A2000C52100086D210008712100088921000896
:106A3000912100089D210008A1210008A52100083E
:106A4000CD21000800000000000000005D220008C9
:106A5000A9210008AD21000800000000000000008E
:106A600051250008592500083D2500084525000846
:106A7000692500086D250008286E756C6C290000DA
:106A800000000000ED290008C5290008752900084C
:106A900091290008AD2900084D444D4120666169E7
:106AA0006C75726500000000009600000000000098
:106AB00000000000000000000000000000000000D6
:106AC00000000000593100084531000881310008FC
:106AD0006D31000879310008653100085131000836
:106AE0003D3100088D3100080000000071320008BF
:106AF0005D320008993200088532000891320008A2
:106B00007D3200086932000855320008A5320008BD
:106B100000000000010000000000000063300000E1
:106B20001C6B0008E8290020F82B002043756265E3
:106B300050696C6F7400437562655265642D424CF8
:106B4000002553455249414C250000000200000039
:106B500000000000913400080135000840004000AA
:106B6000A8440020B84400200200000000000000FB
:106B7000030000000000000049350008000000008C
:106B800010000000C84400200000000001000000C8
:106B900000000000B8480020010102006D4200081A
:106BA0007D41000819420008FD4100084300000033
:106BB000B46B000809024300020100C0320904005E
:106BC000000102020100052400100105240100015A
:106BD000042402020524060001070582030800FFC1
:106BE00009040100020A000000070501024000003C
:106BF000070581024000000012000000006C000840
:106C00001201100102000040AE2D591000020102D5
:106C1000030100000403090425424F4152442500AA
:106C2000437562655265645072696D6172790030B6
:106C300031323334353637383941424344454600E2
:106C400000000020000002000200000000010030EF
:106C50000000000008000000000000240000080000
:106C6000040000000004000000FC0000020000001E
:106C70000000043000800000080000000000003820
:106C8000000001000100000040000052800000529E
:106C9000C000005200010052400100528001005229
:106CA000C001005200020052400200528002005215
:106CB000C002005200030052400300528003005201
:106CC000C00300520004005200000000A536000876
:106CD0005D390008093A000840004000F0490020F2
:106CE000F049002001000000004A00208000000060
:106CF000400100000800000000010000001000003A
:106D0000080000006D61696E0069646C6500000038
:106D10000000802A00000000AAAAAAAA00000024FD
:106D2000FFFF00000000000000A00A00200020007B
:106D300000000000AAAAAAAA00000000FFFF0000AD
:106D40000009000000090000000000000000000031
:106D5000AAAAAAAA00000000FFFF0000000000008D
:106D6000000000000028800A00000000AAAAAAAAC9
:106D700000140000FFFF0000000070070090990061
:106D80002000000000000000AAAAAAAA000000003B
:106D9000FFFF0000000900000000000010000000DC
:106DA00000000000AAAAAAAA00000000FBFF000041
:106DB00000000000000000000104000000000000CE
:106DC000AAAAAAAA00000000FEFF0000000000001E
:106DD000000000000000000000000000AAAAAAAA0B
:106DE00000000000FFFF00000000000000000000A5
:106DF0000000000000000000AAAAAAAA00000000EB
:106E0000FFFF000000000000000000000000000084
:106E100000000000AAAAAAAA00000000FFFF0000CC
:106E20000000000000000000000000000000000062
:106E3000AAAAAAAA00000000FFFF000000000000AC
:106E400000000000DC94FF7F010000000000000053
:106E50002D0400000000000000001A0000000002E5
:106E6000FF000000002C002024250020000000006E
:106E700040680008830400004B68000850040000CC
:106E80005968000800960000000008009600000005
:106E90000008000004000000146C0008000000005E
:106EA00000000000000000000000000000000000E2
:106EB0000000000068220020000000000000000028
:106EC00000000000000000000000000000000000C2
:106ED00000000000000000000000000000000000B2
:106EE00000000000000000000000000000000000A2
:106EF0000000000000000000000000000000000092
:106F00000000000000000000000000000000000081
:086F1000000000000000000079
:00000001FF
